:100000000C94D5030C94F2030C94F2030C942B285B
:100010000C942B310C94F2030C94F2030C94F20325
:100020000C94F2030C94F2030C94F2030C94171C3E
:100030000C94F2030C94F2030C94F2030C94F2036C
:100040000C94D7140C94F2030C9410130C94CB1250
:100050000C94F2030C94F2030C94F2030C94F2034C
:100060000C94F2030C94F203C51FCC1FCF1FD21FB8
:10007000D71FE11FED1F6B206B206B20F71FF91FAF
:1000800002200B2015206B206B206B206B206B2037
:100090001F202D203B204520482051205A205F2042
:1000A000084AD73B3BCE016E84BCBFFDC12F3D6CDF
:1000B00074319ABD56833DDA3D00C77F11BED9E445
:1000C000BB4C3E916BAAAABE000000803F05A84C25
:1000D000CDB2D44EB93836A9020C50B991868808F1
:1000E0003CA6AAAA2ABE000000803F3E0D0A002CB2
:1000F00052583A002C4275663A002C002C57506F2B
:10010000733A002C002C4D506F733A003C436865E5
:10011000636B003C416C61726D003C486F6D650023
:100120003C486F6C64003C52756E003C51756575BF
:1001300065003C49646C65005D0D0A005B302E393A
:10014000672D44726F704C69742E32303134303800
:1001500032353A000D0A003D00244E005D0D0A00C4
:10016000204600205400204D3800204D3900204DFD
:100170003500204D3400204D3300204D3200204DFD
:100180003100204D300020473934002047393300FA
:1001900020473931002047393000204732300020D5
:1001A000473231002047313900204731380020479D
:1001B0003137002047005B473830005B4733005B36
:1001C0004732005B4731005B4730005D0D0A005B42
:1001D000544C4F3A005D0D0A002C005B4739323A0F
:1001E000005D0D0A002C003A003330003238005B0D
:1001F00047005D0D0A002C005B5052423A00290D69
:100200000A00206D61782074726176656C2C206D17
:100210006D0020616363656C2C206D6D2F736563C9
:100220005E3200206D617820726174652C206D6DE6
:100230002F6D696E002C20737465702F6D6D007AC0
:1002400000790078002028003D0024002028686FF5
:100250006D696E672070756C6C2D6F66662C206DF5
:100260006D290D0A002028686F6D696E672064652E
:10027000626F756E63652C206D736563290D0A24AA
:1002800032373D002028686F6D696E6720736565A1
:100290006B2C206D6D2F6D696E290D0A2432363D51
:1002A000002028686F6D696E6720666565642C2084
:1002B0006D6D2F6D696E290D0A2432353D00290DB3
:1002C0000A2432343D002028686F6D696E6720640F
:1002D000697220696E76657274206D61736B3A0085
:1002E0002028686F6D696E67206379636C652C20C8
:1002F000626F6F6C290D0A2432333D00202868613B
:100300007264206C696D6974732C20626F6F6C2944
:100310000D0A2432323D002028736F6674206C6908
:100320006D6974732C20626F6F6C290D0A24323151
:100330003D0020286175746F2073746172742C20E5
:10034000626F6F6C290D0A2432303D0020287265DF
:10035000706F727420696E636865732C20626F6FB2
:100360006C290D0A2431343D002028617263207409
:100370006F6C6572616E63652C206D6D290D0A24AA
:1003800031333D0020286A756E6374696F6E206496
:100390006576696174696F6E2C206D6D290D0A2474
:1003A00031323D00290D0A2431313D00202873747B
:1003B00061747573207265706F7274206D61736BF8
:1003C0003A00202870726F62652070696E20696E35
:1003D000766572742C20626F6F6C290D0A2431309F
:1003E0003D0020286C696D69742070696E73206906
:1003F0006E766572742C20626F6F6C290D0A24363C
:100400003D0020287374657020656E61626C652004
:10041000696E766572742C20626F6F6C290D0A24E8
:10042000353D00290D0A24343D00202864697220DE
:10043000706F727420696E76657274206D61736B73
:100440003A00290D0A24333D00202873746570207A
:10045000706F727420696E76657274206D61736B53
:100460003A002028737465702069646C65206465A7
:100470006C61792C206D736563290D0A24323D006F
:100480002028737465702070756C73652C207573EB
:100490006563290D0A24313D0024303D00242420C9
:1004A0002876696577204772626C20736574746979
:1004B0006E6773290D0A2423202876696577202327
:1004C00020706172616D6574657273290D0A24472D
:1004D0002028766965772070617273657220737465
:1004E000617465290D0A24492028766965772062A0
:1004F00075696C6420696E666F290D0A244E202888
:1005000076696577207374617274757020626C6FA0
:10051000636B73290D0A24783D76616C756520281C
:1005200073617665204772626C2073657474696EBE
:1005300067290D0A244E783D6C696E652028736129
:100540007665207374617274757020626C6F636B72
:10055000290D0A24432028636865636B2067636F55
:100560006465206D6F6465290D0A245820286B6925
:100570006C6C20616C61726D206C6F636B290D0A6D
:100580002448202872756E20686F6D696E6720633D
:1005900079636C65290D0A7E20286379636C652078
:1005A0007374617274290D0A2120286665656420C0
:1005B000686F6C64290D0A3F202863757272656E3E
:1005C0007420737461747573290D0A6374726C2DD1
:1005D0007820287265736574204772626C290D0A51
:1005E000000D0A4772626C20302E39672D44726FFD
:1005F000704C6974205B27242720666F7220686521
:100600006C705D0D0A005D0D0A0044697361626CD7
:10061000656400456E61626C656400436175746970
:100620006F6E3A20556E6C6F636B656400272448CB
:10063000277C2724582720746F20756E6C6F636B9E
:1006400000526573657420746F20636F6E74696EF9
:100650007565005B000D0A0050726F62652066616F
:10066000696C0041626F727420647572696E6720F4
:100670006379636C6500486172642F736F667420E0
:100680006C696D697400414C41524D3A20000D0A6D
:1006900000496E76616C69642067636F6465204908
:1006A000443A00556E646566696E656420666565EA
:1006B00064207261746500556E737570706F72742A
:1006C000656420636F6D6D616E64004D6F64616C75
:1006D0002067726F75702076696F6C6174696F6ED8
:1006E000004C696E65206F766572666C6F770048A6
:1006F0006F6D696E67206E6F7420656E61626C65E8
:100700006400416C61726D206C6F636B004E6F749E
:100710002069646C6500454550524F4D20726561FB
:1007200064206661696C2E205573696E672064656C
:100730006661756C74730056616C7565203C20337E
:1007400020757365630053657474696E672064690E
:100750007361626C65640056616C7565203C203085
:1007600000496E76616C69642073746174656D65AF
:100770006E7400426164206E756D62657220666FF2
:10078000726D617400457870656374656420636F91
:100790006D6D616E64206C65747465720065727253
:1007A0006F723A20006F6B0D0A0011241FBECFEF4D
:1007B000D8E0DEBFCDBF11E0A0E0B1E0EEE7FEE69D
:1007C00002C005900D92A030B107D9F716E0A0E065
:1007D000B1E001C01D92A73CB107E1F70E94F4030C
:1007E0000C943D370C9400001F930E9498120E94B5
:1007F00073210E94ED140E941A318EE1E7E2F5E0C8
:10080000DF011D928A95E9F781E0809327057894AE
:1008100011E00E940B130E9447120E945B120E947B
:1008200077120E94A5270E94DA2B0E94A9260E9417
:10083000E71B0E942D220E948D081092270510921E
:1008400029058091B60681FF03C01093370502C0C9
:10085000109237050E943314DCCF8091290584FD66
:100860001AC08FB7F894909129059061909329054B
:100870008FBF0E945F120E947A12809128058473B4
:1008800051F09FB7F89480912905806280932905E3
:100890009FBF0E94BB1B089584E0809328050E949F
:1008A000C92784E00E945F280E9476138091270563
:1008B000882341F40E948D08109228050E94BB1BDA
:1008C0000E94A5270895EF92FF920F931F93CF9355
:1008D000DF937B018C0180912805823009F447C0A9
:1008E000C801B70120E030E040EA51E40E9416362A
:1008F0000E94AA340E944134EB010E941014C801E6
:10090000B70120E030E04AE754E40E9416367B014C
:100910008C0182E390E0C89FB001C99F700DD89F01
:10092000700D112480E090E00E946D349B01AC01B9
:10093000C801B7010E94F3320E94AA340E944134D8
:10094000DC01CB010E94722700E911E00EC00E9479
:10095000761380912705882351F484EF91E0F80104
:100960003197F1F70197D9F72197209781F7DF9118
:10097000CF911F910F91FF90EF900895DF92EF922A
:10098000FF920F931F93CF93DF93EC017A018B01BA
:10099000D22E8091B60685FF03C0CE010E94D427D7
:1009A000809128058230D1F00E947613809127052E
:1009B0008823A1F40E942322882319F00E9469133E
:1009C000F3CFCE01B801A7012D2D0E94B323809152
:1009D0002805882319F488E080932805DF91CF91BA
:1009E0001F910F91FF90EF90DF9008956F927F928B
:1009F0008F929F92AF92BF92CF92DF92EF92FF922F
:100A00000F931F93CF93DF936C014A015B01722E0A
:100A100080912805823009F489C00E9410146090EA
:100A200037050E94E82B882351F09FB7F8948091F6
:100A300029058064809329059FBF0E9476138091C9
:100A40002705882309F072C0C601B501A401272D2E
:100A50000E94BE0481E0809338059FB7F89480918E
:100A600029058260809329059FBF0E94761380919B
:100A70002705882309F05AC080912805882311F0A2
:100A8000883099F780913805813041F49FB7F89408
:100A9000809129058064809329059FBF0E94761369
:100AA00080912705882309F041C00E94E71B0E941E
:100AB000A9260E942D2289E3E82E85E0F82EC0E0C9
:100AC000D0E086010C0F1D1FF7016191719181919A
:100AD00091917F010E946F34FE01E758F94F208108
:100AE0003181428153810E94D433F8016083718344
:100AF000828393832496CC30D10519F7C601B501C2
:100B0000A401272D0E94BE048FB7F8949091290567
:100B10009260909329058FBF0E9410148091270541
:100B2000882321F4609237050E943D2CDF91CF91FC
:100B30001F910F91FF90EF90DF90CF90BF90AF90FB
:100B40009F908F907F906F9008952F923F924F9239
:100B50005F926F927F928F929F92AF92BF92CF924D
:100B6000DF92EF92FF920F931F93DF93CF93CDB756
:100B7000DEB7EF970FB6F894DEBF0FBECDBF9CABCC
:100B80008BAB7EAB6DAB3A010FAB18AF29AF3AAF71
:100B9000CBAEDCAEEDAEFEAEAFAE9924880C991CA8
:100BA000880C991C880D991D9AAB89AB9A01280D68
:100BB000391D38AB2FA7D901AD90BD90CD90DC90F9
:100BC000C601B501E9A9FAA9208131814281538189
:100BD0000E94F4326DA37EA38FA398A765966FAD94
:100BE0006597462E5524440C551C440C551C2BA9C6
:100BF0003CA9240D351D3EA72DA7C301840D951DCD
:100C00009CA78BA7DC01ED90FD900D911C91C80174
:100C1000B701F90120813181428153810E94F43270
:100C200069A37AA38BA39CA3D601C501B0588D8F6D
:100C30009E8FAF8FB8A3D801C701B058898F9A8F04
:100C4000AB8FBC8FADA9BEA98A0E9B1EF40160813B
:100C50007181828193812DA13EA14FA158A50E944F
:100C6000F3323B014C012DA93EA9420E531ED20185
:100C70006D917D918D919C9129A13AA14BA15CA18F
:100C80000E94F3325B016C016D8D7E8D8F8D98A17A
:100C9000A60195010E9416367B018C01698D7A8D23
:100CA0008B8D9C8DA40193010E9416369B01AC0193
:100CB000C801B7010E94F3321B012C016D8D7E8D9E
:100CC0008F8D98A1A40193010E9416367B018C019F
:100CD000698D7A8D8B8D9C8DA60195010E941636AB
:100CE0009B01AC01C801B7010E94F4329B01AC0129
:100CF000C201B1010E9467335B016C01809145051F
:100D0000823099F4C601B50120E030E040E050E0C7
:100D10000E94DB358823ECF0C601B5012BED3FE0E6
:100D200049EC50E40E94F33212C0C601B50120E044
:100D300030E040E050E00E94CD33181654F0C60178
:100D4000B5012BED3FE049EC50E40E94F4325B0129
:100D50006C01E090B206F090B3060091B4061091D9
:100D6000B5066FA978AD89AD9AAD9B01AC010E9423
:100D7000F432A80197010E94F3329B01AC01C80133
:100D8000B7010E9416360E94A3367B018C01C60172
:100D9000B50120E030E040E05FE30E9416362FA965
:100DA00038AD49AD5AAD0E9416369F77A80197011C
:100DB0000E94D4330E94AA340E944134788F6F8BF2
:100DC0006115710509F487C1BFADBB2381F080E0D7
:100DD00090E00E946D349B01AC016BAD7CAD8DAD9C
:100DE0009EAD0E9416366BAF7CAF8DAF9EAF2F8944
:100DF000388DB90180E090E00E946D347B018C0158
:100E0000C601B501A80197010E94D4336B8B7C8B7E
:100E10008D8B9E8B6696EFAD6697F0E0EE0FFF1F11
:100E2000EE0FFF1F8BA99CA98E0F9F1F9AA789A762
:100E3000ADA9BEA9EA0FFB1F6081718182819381F8
:100E4000E9A5FAA520813181428153810E94F332C4
:100E5000A80197010E94D4336F87788B898B9A8B76
:100E60006B897C898D899E899B01AC010E94163615
:100E70009B01AC0160E070E080E090E40E94F332FE
:100E80005B016C016B897C898D899E892BEA3AEA2A
:100E90004AE25EE30E9416367B018C01C601B50171
:100EA00020E030E040E850E40E94F4329B01AC01C5
:100EB000C801B7010E9416366B877C878D879E8795
:100EC000C601B50120E030E040E05FE30E94163645
:100ED00069837A838B839C8321E030E03E832D837A
:100EE0009924F1C03BE0391508F446C06D8D7E8D24
:100EF0008F8D98A12B853C854D855E850E94163689
:100F00007B018C01698D7A8D8B8D9C8D29813A8135
:100F10004B815C810E9416369B01AC01C801B70170
:100F20000E94F4327B018C016D8D7E8D8F8D98A196
:100F300029813A814B815C810E9416365B016C01EC
:100F4000698D7A8D8B8D9C8D2B853C854D855E853D
:100F50000E9416369B01AC01C601B5010E94F33216
:100F60006D8F7E8F8F8F98A39394C701D801898F3F
:100F70009A8FAB8FBC8F61C0AD81BE81BD0180E017
:100F800090E00E946D342B893C894D895E890E94D6
:100F900016367B018C01C8010E94D1336F8378879C
:100FA00089879A87B701C8010E9499363B014C0195
:100FB000EFA5F8A9E080F1800281138117FB10955D
:100FC00017F91095ABA5BCA52D903D904D905C9068
:100FD000C801B7012F81388549855A850E94163688
:100FE0005B016C01C201B101A40193010E9416369C
:100FF0009B01AC01C601B5010E94F4326D8F7E8F5A
:101000008F8F98A3C801B701A40193010E941636DF
:101010007B018C01C201B1012F81388549855A8538
:101020000E9416369B01AC01C801B7010E94F33241
:10103000698F7A8F8B8F9C8F99246DA17EA18FA150
:1010400098A52D8D3E8D4F8D58A10E94F432E9A9AF
:10105000FAA9608371838283938369A17AA18BA1AA
:101060009CA1298D3A8D4B8D5C8D0E94F432ADA5EB
:10107000BEA56D937D938D939C931397E9A5FAA5D7
:1010800060817181828193812F85388949895A894C
:101090000E94F432A9A5BAA56D937D938D939C937C
:1010A00013978BA99CA94BAD5CAD6DAD7EAD2FADFB
:1010B0000E94BE04809127058823B1F4ED81FE8152
:1010C0003196FE83ED832D813E818F89988D28177F
:1010D000390708F407CF8DA99EA94BAD5CAD6DAD66
:1010E0007EAD2FAD0E94BE04EF960FB6F894DEBF22
:1010F0000FBECDBFCF91DF911F910F91FF90EF9069
:10110000DF90CF90BF90AF909F908F907F906F9027
:101110005F904F903F902F90089560912B057091B4
:101120002C0580912D0590912E050E946F34209101
:10113000790630917A0640917B0650917C060E9498
:10114000D433609358057093590580935A05909352
:101150005B0560912F05709130058091310590916C
:1011600032050E946F3420917D0630917E064091B9
:101170007F06509180060E94D43360935C05709383
:101180005D0580935E0590935F05609133057091D6
:10119000340580913505909136050E946F34209179
:1011A00081063091820640918306509184060E9408
:1011B000D4336093600570936105809362059093CA
:1011C000630508952F923F924F925F926F927F92A4
:1011D0008F929F92AF92BF92CF92DF92EF92FF9247
:1011E0000F931F93DF93CF93CDB7DEB7A8970FB6BA
:1011F000F894DEBF0FBECDBF1C01E0E8F5E089E347
:10120000DF011D928A95E9F73196A5E4B5E08AE001
:101210000D9001928150E1F7198277246624AA2467
:10122000BB241F8E1E8E1CA261E0462E512C9924D9
:10123000939452E0852E6BC2802F81548A3118F02E
:1012400081E00C942E129F5F9983C101BE016F5FF4
:101250007F4FAE014E5F5F4F0E94BA26882319F47C
:1012600082E00C942E12CA80DB80EC80FD80C701E6
:10127000B6010E94F0360E944134162F70E0882794
:1012800077FD8095982F0E946F349B01AC01C701B8
:10129000B6010E94F33220E030E048EC52E40E94B4
:1012A00016360E9479360E944134262F073421F0E9
:1012B0000D3409F053C10BC1163209F496C0173230
:1012C000F0F4143170F4113108F0BAC0143009F49C
:1012D00043C0143008F489C01A3011F00C941D1268
:1012E00032C01C3181F11D3128F4163110F00C94FC
:1012F0001D12C8C01E3111F00C941D1224C01035EF
:1013000009F47AC0113588F4153331F1163340F4FD
:101310001B3209F4C0C0113311F00C941D12BBC074
:101320001C3310F00C941D12CBC01C3561F01D3520
:1013300028F41A3510F40C941D1292C01F3510F0C9
:101340000C941D1296C0222339F4BCA1BB2311F0CA
:101350000C941B12E1E0ECA31C31A9F01D3128F420
:10136000143051F01A3069F40AC0153351F11C35AC
:1013700061F11E3131F416C09092800502C0809256
:10138000800580E0A1C0222329F02A3011F00C94BE
:101390001D1204C0F3E0F093800521C024E02093E7
:1013A00080051DC0222329F02A3011F00C941D1253
:1013B00004C085E08093800512C096E0909380057C
:1013C0000EC0A7E0A0938005DCCF222329F02A30AD
:1013D00011F00C941D1205C0B8E0B093800580E0B8
:1013E000AEC0E9E0E0938005FACFFCA1FF2311F045
:1013F0000C941B1282E08CA3123089F0133028F475
:10140000112351F01130D1F40AC0163259F01035C1
:1014100091F0133099F403C0109281050FC010931E
:1014200081050CC0243111F00C941D1294E09093AE
:10143000810581E084C0A5E0A093810581E044C0DE
:10144000123139F0133149F0113129F41092850528
:1014500002C09092850582E037C080928505FBCF5F
:101460001A3519F41092840502C09092840583E025
:101470002BC01D3519F49092820502C0109282058E
:1014800084E022C0143119F49092830502C01092B6
:10149000830585E019C0BCA1BB2309F0CCC711337B
:1014A00031F41092860586E0E3E0ECA348C02A30D0
:1014B00009F0C3C79092860586E0F3E0FCA33FC025
:1014C00016531093870587E02223C9F1B8C7662316
:1014D00009F0B5C7163018F41330B0F408C018304E
:1014E00008F4ABC71A3000F11E3109F0A6C712305C
:1014F00041F01E3131F0112311F49092880588E0FB
:101500001EC080928805FBCF143039F0153041F0B1
:10151000133041F490928A0505C080928A0502C07A
:1015200010928A0589E00BC0183019F0193031F497
:1015300003C08092890502C0109289058AE0920159
:1015400002C0220F331F8A95E2F7C9018A219B212D
:10155000892B09F076C7A22AB32AD9C0003509F42D
:101560006BC001359CF40A34E9F10B3434F40634D1
:1015700021F1093409F061C72AC00C3409F44AC0CA
:101580000C34E4F10E3409F058C748C0043599F022
:1015900005353CF4023509F459C0033509F04DC74F
:1015A0005FC0093509F472C00A3509F47BC00835FB
:1015B00009F043C75FC029E080C0C0928B05D0927C
:1015C0008C05E0928D05F0928E0520E076C0C092E9
:1015D0008F05D0929005E0929105F092920521E05E
:1015E000622A6BC0C0929305D0929405E092950553
:1015F000F092960582E0682A22E05FC0C0929705CB
:10160000D0929805E0929905F0929A0594E0692AA3
:1016100023E053C010939B0524E04FC0C701B601DF
:101620000E943C3460939C0570939D0580939E05B9
:1016300090939F0525E041C0C092A005D092A105DE
:10164000E092A205F092A30526E037C0C092A4055F
:10165000D092A505E092A605F092A70527E02DC03F
:10166000C092A805D092A905E092AA05F092AB0518
:1016700028E023C0C092AD05D092AE05E092AF0540
:10168000F092B005A1E07A2A2AE017C0C092B10515
:10169000D092B205E092B305F092B405B2E07B2A95
:1016A0002BE00BC0C092B505D092B605E092B7050D
:1016B000F092B805E4E07E2A2CE08201022E02C0FE
:1016C000000F111F0A94E2F78E8D9F8D80239123C6
:1016D000892B11F089E1C2C681E693E002C095959D
:1016E00087952A95E2F780FF0CC0C701B60120E07C
:1016F00030E040E050E00E94CD33882314F484E0D1
:10170000ADC68E8D9F8D802B912B9F8F8E8F998153
:10171000F101E90FF11D0081002309F08DCD772043
:1017200029F09CA1992311F4A2E0ACA3BE8DB5FFD2
:101730000FC080919C0590919D05A0919E05B09150
:101740009F0580589649A849B04014F08BE186C6A1
:1017500080918205813039F4FCA1F230B1F52E8DF3
:1017600020FD33C070C680914605882371F58E8DAB
:1017700080FF1BC080918305813039F560918B0516
:1017800070918C0580918D0590918E0523E333E354
:101790004BEC51E40E94163660938B0570938C05D8
:1017A00080938D0590938E0510C080915305909184
:1017B0005405A0915505B091560580938B059093E3
:1017C0008C05A0938D05B0938E05AE8DBF8DB0FDB9
:1017D00010C080914F0590915005A0915105B09196
:1017E00052058093A8059093A905A093AA05B093EC
:1017F000AB0580918005813041F4BE8DB6FF25C6D2
:10180000EE8DFF8DEF7BFF8FEE8F80918505882316
:1018100041F0813061F4F2E0FBA31AA221E029A398
:101820000BC01BA281E08AA392E099A305C0A1E0AE
:10183000ABA3B2E0BAA319A280918305813059F518
:101840004DEAE42E45E0F42E00E010E0C72CDD2444
:10185000C601002E02C0959587950A94E2F780FF95
:1018600011C0F701608171818281938123E333E3A9
:101870004BEC51E40E941636D7016D937D938D9306
:101880009C9313970F5F1F4FE4E0F0E0EE0EFF1EF6
:1018900003301105E9F6FCA1F33049F48091860587
:1018A000813029F424E0721611F085E2D7C5DE01FB
:1018B0001696E4E6F5E08CE001900D928150E1F798
:1018C000A7FE12C090918705973008F0C0C580919F
:1018D0004B05891749F0892FBE016A5F7F4F0E942F
:1018E0004821882309F4B5C580918005823021F014
:1018F000883009F0FDC09AC0772009F4ACC58E8D00
:101900009F8D80759070892B09F49FC56091A0050B
:101910007091A1058091A2059091A3050E94F036D7
:101920000E944134673008F092C520919B05243114
:1019300031F0223009F081C58E8D87FD7EC566238A
:1019400019F0615068A303C09091870598A38E0198
:101950000E5E1F4F88A1B8010E944821882309F418
:1019600078C578013DEA832E35E0932E28E5C22E16
:1019700025E0D22E00E010E0A72CBB24C501002EEC
:1019800002C0959587950A94E2F780FF3BC080914D
:101990009B05843169F5D6016D917D918D919C9166
:1019A000139758962D913D914D915C915B970E94B4
:1019B000F332F40120813181428153810E94F3325C
:1019C000D7016D937D938D939C9313970230D1F43F
:1019D00020917C0530917D0540917E0550917F05D9
:1019E0000E94F332F70160837183828393830AC07C
:1019F000F40180819181A281B381F7018083918379
:101A0000A283B3830F5F1F4F84E090E0E80EF91EBE
:101A1000880E991EC80ED91E0330110509F0AECFED
:101A2000AE8DBF8DAF7ABF8FAE8F02C1772009F424
:101A300012C50DEA15E098E5C92E95E0D92E86E08D
:101A4000882E912C8C0E9D1EEE24FF24A72CBB24E7
:101A5000C5010E2C02C0959587950A94E2F780FF88
:101A60002CC0F6016081718182819381D4012D9116
:101A70003D914D915C910E94F332F80120813181BA
:101A8000428153810E94F332D8016D937D938D93EF
:101A90009C931397B2E0EB16D1F420917C05309122
:101AA0007D0540917E0550917F050E94F332F8013B
:101AB00060837183828393830AC0F601808D918D48
:101AC000A28DB38DF80180839183A283B3830894A0
:101AD000E11CF11C0C5F1F4F84E090E0C80ED91E82
:101AE000880E991E93E0E916F10409F0B1CF9FC06A
:101AF000ACA1A33009F47CC0772009F479C018E5C3
:101B0000C12E15E0D12E0DEA15E0B6E0AB2EB12CBA
:101B1000AC0EBD1EEE24FF24872C9924C4010E2C8C
:101B200002C0959587950A94E2F780FD0BC0F601F7
:101B300080819181A281B381F80180839183A28306
:101B4000B38346C080918005873009F441C08091FD
:101B50008405882361F5D5016D917D918D919C91CE
:101B6000F601208D318D428D538D0E94F432D801C3
:101B70002D913D914D915C910E94F432F80160836A
:101B8000718382839383F2E0EF1611F520917C0537
:101B900030917D0540917E0550917F050E94F43281
:101BA000D8016D937D938D939C93139711C0F80189
:101BB0006081718182819381D6012D913D914D91FA
:101BC0005C910E94F432F801608371838283938375
:101BD0000894E11CF11C84E090E0C80ED91E0C5F53
:101BE0001F4FA80EB91E93E0E916F10409F096CF35
:101BF00080918005853049F0873099F08330B9F4C1
:101C0000772009F41CA286E004C0772009F41CA206
:101C100087E0BE016E5E7F4F0E944821882339F421
:101C200018C480918105823010F08EE117C418A28B
:101C300010918105153049F4772009F45FC2ACA1F9
:101C4000A13009F45BC28FE109C4BCA1B23009F034
:101C500055C21123E9F060918B0570918C0580913C
:101C60008D0590918E0520E030E040E050E00E942C
:101C7000CD33882309F4E7C3143030F4123060F414
:101C8000113009F03BC204C0143009F037C213C24E
:101C9000772009F432C232C2772009F4DCC3FBA1F9
:101CA000EF2FF0E0F8A7EFA39AA1892F90E09EA371
:101CB0008DA381E090E08C010DA002C0000F111FE8
:101CC0000A94E2F70FA002C0880F991F0A94E2F766
:101CD000082B192B872D90E080239123892B11F459
:101CE00080E2BCC3EFA1F8A5EE0FFF1FEE0FFF1FB0
:101CF000DF01AB5BBA4FE058FA4F65A576A587A523
:101D000090A953962D913D914D915C9156970E94CB
:101D1000F3325B016C01EDA1FEA1EE0FFF1FEE0F90
:101D2000FF1FDF01AB5BBA4FE058FA4F65A576A500
:101D300087A590A953962D913D914D915C91569711
:101D40000E94F3321B012C01AE8DA7FF02C108E5F2
:101D500015E06DEAE62E65E0F62EF80160817181EE
:101D600082819381D7012D913D914D915C910E948B
:101D7000CD33882359F40C5F1F4FE4E0F0E0EE0E02
:101D8000FF1EF5E004361F0741F767C38091830506
:101D90008130B1F46091A4057091A5058091A605EC
:101DA0009091A70523E333E34BEC51E40E941636F0
:101DB0006093A4057093A5058093A6059093A7054D
:101DC000E090A405F090A5050091A6051091A70547
:101DD000C801B70120E030E040E850E40E94163628
:101DE000A80197010E9416367B018C01C601B5013E
:101DF000A60195010E9416369B01AC01C801B701EE
:101E00000E94F3327B018C01C201B101A201910158
:101E10000E9416369B01AC01C801B7010E94F33243
:101E20007B018C0120E030E040E050E00E94CD33A7
:101E3000882314F482E212C3C801B7010E94A336BA
:101E40007B018C01C601B501A20191010E947C2792
:101E50009B01AC0117FB109517F91095C801B7014C
:101E60000E94D4337B018C0180918105833021F461
:101E700017FB109517F910956090A4057090A505B3
:101E80008090A6059090A705C401B30120E030E042
:101E900040E050E00E94CD3388237CF417FB10957E
:101EA00017F91095D401C301B0588093A4059093FD
:101EB000A505A093A605B093A7058E8D9F8D8F775E
:101EC0009F8F8E8FAFA1B8A5AA0FBB1FAA0FBB1FF4
:101ED000AC57BA4FB8A7AFA3C201B101A80197018F
:101EE0000E9416369B01AC01C601B5010E94F33277
:101EF00020E030E040E05FE30E941636EFA1F8A555
:101F000063877487858796878DA19EA1880F991F07
:101F1000880F991F8C579A4F9EA38DA3C601B501B8
:101F2000A80197010E9416369B01AC01C201B101C4
:101F30000E94F43220E030E040E05FE30E94163679
:101F4000ADA1BEA11B966D937D938D939C931E971F
:101F5000D5C0862C992408211921012B11F483E284
:101F60007DC2EE8DFF8DE17FFF8FEE8F8091830527
:101F7000813041F53FE8E32E35E0F32E00E010E03C
:101F8000C401002E02C0959587950A94E2F780FF60
:101F900010C0D7016D917D918D919C9123E333E326
:101FA0004BEC51E40E941636F70160837183828303
:101FB00093830F5F1F4F84E090E0E80EF91E03301B
:101FC0001105F1F6EFA0F8A4EE0CFF1CEE0CFF1CBF
:101FD000A4E8B5E0EA0EFB1EC601B501F7012385B2
:101FE0003485458556850E94F3325B016C010DA155
:101FF0001EA1000F111F000F111F0C571A4FC20115
:10200000B101D8011B962D913D914D915C911E9788
:102010000E94F3329B01AC01C601B5010E947C27EE
:102020005B016C01F7016385748585859685D80110
:102030001B962D913D914D915C911E970E947C279E
:102040003B014C016093A4057093A5058093A60500
:102050009093A705C601B501A40193010E94F33234
:102060007B018C01E89417F9C801B7012AE037ED2C
:1020700043EA5BE30E94DB3518160CF03FC0C80151
:10208000B70120E030E040E05FE30E94DB35181646
:102090000CF4E3C1C401B3012FE632E143E85AE393
:1020A0000E9416369B01AC01C801B7010E94DB35C6
:1020B000181624F5D2C1772009F4CDC108E515E042
:1020C0008DEAE82E85E0F82EF80160817181828129
:1020D0009381D7012D913D914D915C910E94CD331B
:1020E000882361F40C5F1F4FE4E0F0E0EE0EFF1E6A
:1020F000F5E004361F0741F7B0C11CA28E8D9F8DFD
:102100008E7D9C7F2CA1222321F08E8D9F8D8E7D34
:10211000907E892B11F084E2A1C180918205809389
:10212000460580918B0590918C05A0918D05B0910D
:102130008E058093530590935405A0935505B09355
:102140005605E090A805F090A9050091AA05109108
:10215000AB0560914F0570915005809151059091AC
:102160005205A80197010E94CD33882381F0E092A7
:102170004F05F09250050093510510935205809140
:102180004E05882321F0B801A7010E9461128091B9
:10219000AC058093570590918A0580914E0589176B
:1021A00069F090934E0540914F0550915005609114
:1021B000510570915205892F0E94611290918905F5
:1021C00080914D05891729F090934D05892F0E9424
:1021D0007C1280918005813051F46091A00570914E
:1021E000A1058091A2059091A3050E9463048091AE
:1021F00085058093490580918305809347058CA1CF
:102200008330D9F48091860580934A05813049F462
:102210008091B5059091B605A091B705B091B8052C
:1022200004C080E090E0A0E0B0E080937C05909353
:102230007D05A0937E05B0937F05909187058091E1
:102240004B05891759F090934B05A4E6B5E0FE01C4
:1022500036968CE001900D928150E1F780918405D3
:102260008093480580918005853059F1863048F487
:10227000833039F1843008F044C0823009F05AC00C
:102280000AC0883009F445C0893009F44CC0863052
:1022900009F050C038C08E010E5E1F4F88A1B801F2
:1022A0000E943D2180914B0598A1891709F042C0F9
:1022B000A4E6B5E0F8018CE001900D928150E1F7C1
:1022C00039C0ACA1AA2349F08DEA95E040E050E086
:1022D00060E87FEB20E00E94BE048E010E5E1F4F7F
:1022E000C80140E050E060E87FEB20E00E94BE04BF
:1022F000A8E5B5E0F8018CE001900D928150E1F77E
:1023000019C086E001C087E068E575E00E943D21C4
:1023100011C0A0E7B5E0EDEAF5E08CE001900D9288
:102320008150E1F707C08CE0E0E7F5E0DF011D92A6
:102330008A95E9F78091810580934505853009F4F8
:1023400065C0BCA1B23009F061C0843040F4823075
:1023500008F5882341F0813009F04FC00CC084306B
:1023600009F04BC03CC08DEA95E040E050E060E8E9
:102370007FEB20E00CC040915305509154056091D3
:102380005505709156058DEA95E0209146050E940D
:10239000BE0433C000D00091A4051091A505209182
:1023A000A6053091A705C0905305D0905405E09044
:1023B0005505F09056058AA1EDB7FEB7818399A126
:1023C000928388E595E06DEA75E04FE855E0A090CE
:1023D00046058BA00E94A5050F900F900EC040915E
:1023E00053055091540560915505709156058DEA3D
:1023F00095E0209146050E94F604A8E5B5E0EDEAD7
:10240000F5E08CE001900D928150E1F78091880514
:1024100080934C05882311F10E9410141092370507
:1024200080914C05823019F40E942D0402C0109254
:102430004C0580E013C088E111C084E10FC087E142
:102440000DC085E10BC086E109C08CE107C08DE1BC
:1024500005C087E003C08AE101C081E2A8960FB6FB
:10246000F894DEBF0FBECDBFCF91DF911F910F91CA
:10247000FF90EF90DF90CF90BF90AF909F908F90A4
:102480007F906F905F904F903F902F900895E5E47C
:10249000F5E08BE3DF011D928A95E9F780914B050A
:1024A000BF01615E7F4F0E944821882319F487E0B5
:1024B0000E94722C0895249A259A2C9808952C989D
:1024C00008951F93182F80912805823071F00E9483
:1024D00069130E941014112311F42C9806C01130B6
:1024E00011F42D9801C02D9A2C9A1F9108953B9AB2
:1024F00043980895439808951F93182F80912805B5
:10250000823049F00E9469130E941014123011F4B5
:10251000439A01C043981F910895909101018091C1
:102520000001891710F0891B08958058891B0895B0
:10253000E0ECF0E08081826080831092C50080E151
:102540008093C400E1ECF0E0808180618083808131
:10255000886080838081806880830895282FE0913F
:1025600002019E2F9F5F903431F490E004C080916F
:10257000290584FD0FC0809103019817C1F3F0E095
:10258000E754FA4F2083909302018091C10080624A
:102590008093C10008951F920F920FB60F921124DD
:1025A0008F939F93EF93FF9380910301E82FF0E0C7
:1025B000E754FA4F90819093C600982F9F5F903414
:1025C00009F490E09093030180910201981729F497
:1025D0008091C1008F7D8093C100FF91EF919F9109
:1025E0008F910F900FBE0F901F9018959091010141
:1025F00080910001891711F48FEF0895E92FF0E021
:10260000E750FA4F8081E92FEF5FE03809F4E0E00E
:10261000E0930101089580910001809301010895E4
:102620001F920F920FB60F9211242F933F934F9347
:102630005F936F937F938F939F93AF93BF93EF932A
:10264000FF932091C6002132C9F0223218F42831BC
:10265000F1F41AC02F3319F02E37C9F406C09FB712
:10266000F89480912905816005C09FB7F894809106
:1026700029058260809329059FBF1AC09FB7F894EF
:10268000809129058860F6CF0E942D0411C0E09149
:1026900000019E2F9F5F903809F490E08091010126
:1026A000981731F0F0E0E750FA4F20839093000143
:1026B000FF91EF91BF91AF919F918F917F916F911A
:1026C0005F914F913F912F910F900FBE0F901F90F0
:1026D000189580913705882341F09FB7F894809131
:1026E00029058260809329059FBF0895CF93DF93CA
:1026F00080912905882309F48AC0C82FD0E0CE0133
:1027000080769070892B39F181E080932805C6FF8F
:1027100017C0C5FF02C08FEF01C08DEF0E94F930D6
:1027200081E00E94132C9FB7F894809129058F7E39
:10273000809329059FBF8091290584FFFCCF03C0AA
:102740008EEF0E94F9309FB7F894809129058F7918
:10275000809329059FBFC4FF04C081E080932705B3
:102760005CC0C0FF0AC00E94D92C9FB7F89480912A
:1027700029058E7F809329059FBFC3FF15C08091D7
:102780002805803149F480E2809328050E940F15C6
:102790000E943115109237059FB7F8948091290552
:1027A000877F809329059FBFC1FF1DC080912805A9
:1027B000883089F480E1809328050E9431150E94B9
:1027C000AF148091B60681FF04C081E08093370585
:1027D00002C0109237059FB7F894809129058D7F2C
:1027E000809329059FBFC2FF12C00E941222892B2D
:1027F00021F088E08093280502C0109228059FB739
:10280000F894809129058B7F809329059FBF809143
:102810002805847311F00E943115DF91CF9108953E
:1028200080913705882341F09FB7F894809129055E
:102830008260809329059FBF80912805803151F4E3
:1028400081E08093370506C00E94761380912705AA
:10285000882341F40E941222892BB1F78091280528
:10286000803191F308950F931F930E940E2C809155
:102870002805813021F482E00E94132C1CC01092A4
:10288000280584E091E00E94673115C09A3011F06C
:102890009D3029F5E12FF0E0EC5FFE4F10820E94A1
:1028A000761380912705882331F4809104018823D1
:1028B00021F40E94722C00E025C0843229F484E0C7
:1028C00091E00E949331F5CF80912805813011F479
:1028D00089E0EFCF84E091E00E94E208EACF002394
:1028E00021F0993209F500E01FC09132E8F09F32E3
:1028F000D9F0983211F401E017C01F3428F08BE0B2
:102900000E94722C10E010C0892F8156A12FB0E0D8
:10291000E12FEF5F8A3120F4AC5FBE4F905202C0CE
:10292000AC5FBE4F9C931E2F0E94F612982F8F3FD4
:1029300009F0ACCF80913705882341F09FB7F89418
:10294000809129058260809329059FBF0E9476139C
:1029500080912705882341F31F910F91089580915D
:10296000B60682FF02C0289A01C0289880912805E7
:102970008471E1F08091F4018093DC018091F30196
:102980008093DB018091A90690E0A0E0B0E002977F
:10299000A109B109880F991FAA1FBB1F81958093B8
:1029A000DA0180916F00826080936F0008951F921A
:1029B0000F920FB60F9211248F939F939BB180912A
:1029C000F3018C71937E892B8BB915BC9F918F91EC
:1029D0000F900FBE0F901F9018958AB18C618AB925
:1029E000209A8AB1806E8AB9E1E8F0E080818F7E1A
:1029F0008083808188608083E0E8F0E080818C7F44
:102A0000808380818F708083EEE6F0E08081887F14
:102A1000808314BC15BC8081816080830895CF932E
:102A2000DF93C091F601D091F7012097B9F081E0D2
:102A30008093FB0120911102309112024091130208
:102A400050911402CA01B9010E941636698B7A8B23
:102A50008B8B9C8B1092F7011092F601DF91CF9136
:102A600008952F923F924F925F926F927F928F9232
:102A70009F92AF92BF92CF92DF92EF92FF920F930D
:102A80001F93DF93CF93CDB7DEB7E9970FB6F894D6
:102A9000DEBF0FBECDBF13C68091F6019091F70146
:102AA000892B09F07EC20E9412229093F701809335
:102AB000F601892B09F40AC68091FB01882319F0DD
:102AC0001092FB01CAC08091FA018F5F8093FA01D6
:102AD000853011F41092FA01E091FA0121E1E29FB0
:102AE000F0011124EC5AFE4FF093F901E093F80144
:102AF0000091F6011091F701D8018C918083119615
:102B00002D913D914D915C91149793E0220F331FCD
:102B1000441F551F9A95D1F72183328343835483F1
:102B200015962D913D914D915C91189783E0220F60
:102B3000331F441F551F8A95D1F72583368347835A
:102B4000508719962D913D914D915C911C9773E0A2
:102B5000220F331F441F551F7A95D1F721873287E3
:102B6000438754871D962D913D914D915C915097CF
:102B700063E0220F331F441F551F6A95D1F7258745
:102B800036874787508B1D966D917D918D919C91D5
:102B900050970E946D346093FC017093FD01809307
:102BA000FE019093FF01F80125A136A147A150A590
:102BB0000E94D4339B01AC01609300027093010228
:102BC000809302029093030260E070E080EA9FE34A
:102BD0000E94D4336093040270930502809306022E
:102BE0009093070280E090E0A0E0B0E080930802BC
:102BF00090930902A0930A02B0930B0280912805DA
:102C00008032E1F42091190230911A0240911B02A6
:102C100050911C0220931102309312024093130230
:102C200050931402CA01B9010E941636D801519678
:102C30006D937D938D939C9354970FC0F801618998
:102C40007289838994890E94A336609311027093DC
:102C50001202809313029093140280E090E0A0E0AF
:102C6000B0E080930D0290930E02A0930F02B093F8
:102C700010020091F6011091F701D80191968D9103
:102C80009D910D90BC91A02D88AB99ABAAABBBAB2D
:102C900060E070E080E09FE328A939A94AA95BA918
:102CA0000E94D4331B012C0180912805803209F049
:102CB00056C0B2E0B0930C02F801A5A0B6A0C7A020
:102CC000D0A46188728883889488C201B101A4016C
:102CD00093010E9416369B01AC01C601B5010E940A
:102CE000F3327B018C0120E030E040E050E00E94B4
:102CF000CD338823FCF468A979A98AA99BA920E08F
:102D000030E040E050EC0E941636A60195010E948A
:102D100016369B01AC01C401B3010E94F4320E943B
:102D2000A3366093190270931A0280931B0290934A
:102D30001C0237C1E0920D02F0920E0200930F02C6
:102D40001093100280E090E0A0E0B0E080931902C0
:102D500090931A02A0931B02B0931C0222C11092FE
:102D60000C02F80185A196A1A7A1B0A580931D0230
:102D700090931E02A0931F02B09320020E94912301
:102D80005B016C016093190270931A0280931B021D
:102D900090931C02A60195010E9416363B014C013E
:102DA0002091F6013091F70139AF28AFD9019596FE
:102DB0008D919D910D90BC91A02D8B8F9C8FAD8F8F
:102DC000BE8FF9016189728983899489A401930175
:102DD0000E94F3329B01AC01C201B1010E94163680
:102DE0009B01AC016B8D7C8D8D8D9E8D0E94F4328C
:102DF00020E030E040E05FE30E9416367B018C016A
:102E000020E030E040E050E00E94DB3518160CF086
:102E1000B4C0C801B7012B8D3C8D4D8D5E8D0E94D5
:102E2000CD3388230CF095C0A8ADB9AD5D966D91FA
:102E30007D918D919C919097A40193010E94F33212
:102E40009B01AC01C201B1010E94163660932102C0
:102E5000709322028093230290932402A801970189
:102E60000E94CD3388230CF047C0E8ADF9ADE58C66
:102E7000F68C078D10A1C801B7010E94A33660939C
:102E80001502709316028093170290931802A8AD52
:102E9000B9AD5196AD90BD90CD90DC905497C601E0
:102EA000B501A80197010E94CD33882321F4B1E038
:102EB000B0930C0276C0C801B701A60195010E942B
:102EC000F3329B01AC01C201B1010E9416369B0195
:102ED000AC0160911D0270911E0280911F029091C1
:102EE00020020E94F33260931D0270931E028093B1
:102EF0001F029093200255C0E0921D02F0921E0224
:102F000000931F0210932002E0922102F09222020D
:102F10000093230210932402E8ADF9AD21A132A160
:102F200043A154A1CA01B9010E94F432A80197013A
:102F30000E941636A40193010E94F4320E94A33627
:102F400060931502709316028093170290931802F3
:102F500028C0F2E0F0930C028091110290911202CD
:102F6000A0911302B091140280931502909316025F
:102F7000A0931702B093180214C080E090E0A0E084
:102F8000B0E080931D0290931E02A0931F02B093A5
:102F90002002A0921502B0921602C0921702D0929F
:102FA00018028091F101B6E08B9FD0011124A75542
:102FB000BE4FB9AFA8AF8091FA0112968C93E09101
:102FC000F601F091F701FA8FE98F85A196A1A7A1EB
:102FD000B0A58D8B9E8BAF8BB88FBC01CD0120919E
:102FE00004023091050240910602509107020E94AE
:102FF000F3326CA37DA38EA39FA320E030E040E0DA
:1030000050E00E94CD33882344F480E090E0A0E0BB
:10301000B0E08CA39DA3AEA3BFA380911D029091AD
:103020001E02A0911F02B0912002898B9A8BAB8B5C
:10303000BC8B8091150290911602A0911702B0915D
:1030400018028D879E87AF87B88B8091210290915F
:103050002202A0912302B091240289879A87AB872C
:10306000BC8780910D0290910E02A0910F02B09149
:1030700010028D839E83AF83B8878091190290914F
:103080001A02A0911B02B0911C0289839A83AB8320
:10309000BC838091110290911202A0911302B09111
:1030A000140288A399A3AAA3BBA390910C029F8F9B
:1030B000AD88BE88CF88D88C8EE393ECAEEAB9E3B6
:1030C0008CA79DA7AEA7BFA780E090E0A0E0B0E0EE
:1030D00088A799A7AAA7BBA70F2EFEE36F2EF3EC34
:1030E0007F2EFEEA8F2EF9E39F2EF02D9F8D9923E0
:1030F00021F0913009F0B3C080C0C401B301A98DA3
:10310000BA8D91962D913D914D915C9194970E942D
:1031100016367B018C0120E030E040E05FE30E9446
:1031200016369B01AC0168A179A18AA19BA10E94DE
:10313000F4329B01AC01C401B3010E9416369B011D
:10314000AC01C601B5010E94F3325B016C01298913
:103150003A894B895C890E94CD3388230CF040C0AA
:1031600069897A898B899C8929853A854B855C8513
:103170000E94CD33882319F4B2E0BF8F02C0E1E092
:10318000EF8F6D897E898F89988D29893A894B893E
:103190005C890E94F3329B01AC010E94F4327B01F6
:1031A0008C0168A179A18AA19BA12D853E854F85BF
:1031B00058890E94F4329B01AC01C801B7010E94FA
:1031C000D4333B014C01A988BA88CB88DC888D8533
:1031D0009E85AF85B88988A399A3AAA3BBA3B0C0D5
:1031E00068A179A18AA19BA1A80197010E94F4324C
:1031F00068A379A38AA39BA3A3C06D857E858F85D1
:103200009889A40193010E9416369B01AC01C60166
:10321000B5010E94F3327B018C0129853A854B85EB
:103220005C850E94CD3387FD03C05701680188C0CB
:10323000C601B50129853A854B855C850E94F3322C
:103240002D853E854F8558890E94D4333B014C0122
:10325000A984BA84CB84DC8492E09F8F71C0C401BE
:10326000B301A98DBA8D91962D913D914D915C91AF
:1032700094970E9416367B018C0168A179A18AA1DE
:103280009BA1A80197010E94DB351816ACF5C80177
:10329000B70120E030E040E05FEB0E9416369B0172
:1032A000AC0168A179A18AA19BA10E94F4329B0183
:1032B000AC01C401B3010E9416369B01AC01C601EA
:1032C000B5010E94F3321B012C012D813E814F81FB
:1032D00058850E94DB3518167CF468A179A18AA173
:1032E0009BA1A80197010E94F33268A379A38AA346
:1032F0009BA36201510124C0C601B5012D813E810D
:103300004F8158850E94F3329B01AC010E94F43238
:103310007B018C0168A179A18AA19BA129813A81B5
:103320004B815C810E94F4329B01AC01C801B70162
:103330000E94D4333B014C01AD80BE80CF80D88445
:1033400068A579A58AA59BA5A40193010E94F432E2
:1033500068A779A78AA79BA72CA53DA54EA55FA521
:103360000E94CD3388232CF46CA57DA58EA59FA546
:1033700018C0C601B5012CA13DA14EA15FA10E94BC
:10338000DB3518160CF56CA57DA58EA59FA52EE343
:1033900033EC4EEA59E30E94F4326CA77DA78EA766
:1033A0009FA728A539A54AA55BA50E94F3323B013A
:1033B0004C01C601B5012D813E814F8158850E9487
:1033C000DB3518160CF492CE88A199A1AAA1BBA155
:1033D0008093110290931202A0931302B0931402EF
:1033E0009F8D90930C02C601B5012091000230918F
:1033F000010240910202509103020E9416366CAB0A
:103400007DAB8EAB9FAB0E94BA331B012C01609148
:10341000FC017091FD018091FE019091FF010E94DD
:10342000BA333B014C01A20191010E94F3320E9488
:103430004134A8ADB9AD6D937C93672BB1F5809104
:103440002805803291F580E090E0A0E0B0E0809324
:10345000110290931202A0931302B093140280936E
:10346000080290930902A0930A02B0930B022092E3
:10347000FC013092FD014092FE015092FF0100914B
:10348000F6011091F701C201B101209100023091C3
:10349000010240910202509103020E94D433F801CC
:1034A00065A376A387A390A7FEC068A579A58AA582
:1034B0009BA5209108023091090240910A02509187
:1034C0000B020E94F4327B018C01C401B3012CA9D0
:1034D0003DA94EA95FA90E94F3329B01AC01C8012E
:1034E000B7010E94D4337B018C01C201B1012CA928
:1034F0003DA94EA95FA90E94F332A80197010E943D
:103500001636609308027093090280930A02909322
:103510000B02C801B70120EC31EE44E65EE40E94E4
:1035200016360E94BA330E944134AB01BC01403DC3
:10353000F7E05F07F0E06F07F0E07F0728F4A8AD41
:10354000B9AD15961C9233C0403ABFE05B07B0E0BE
:103550006B07B0E07B0728F421E0E8ADF9AD2583E7
:103560000FC040343FE1530730E0630730E073079A
:1035700010F4E2E001C0E3E0A8ADB9AD1596EC931C
:10358000A8ADB9AD15962C911597022E04C076956D
:103590006795579547950A94D2F78D919C9111970D
:1035A00002C0880F991F2A95E2F78D939C934030B3
:1035B000B0E05B07B1E06B07B0E07B0728F4E8AD53
:1035C000F9AD5483438308C0EFEFFFEFA8ADB9AD69
:1035D0001496FC93EE9313978091F2018093F1017E
:1035E0008F5F8093F201863011F41092F201C601D0
:1035F000B5012D813E814F8158850E94DB3518161B
:10360000ACF4E091F601F091F701A5A2B6A2C7A231
:10361000D0A68CA99DA9AEA9BFA98093FC019093C7
:10362000FD01A093FE01B093FF0149C0C601B501A1
:1036300020E030E040E050E00E94DB351816CCF589
:1036400080E090E0A0E0B0E080931102909312023D
:10365000A0931302B093140280930802909309027E
:10366000A0930A02B0930B022092FC013092FD015C
:103670004092FE015092FF010091F6011091F70176
:10368000C201B10120910002309101024091020279
:10369000509103020E94D433D80195966D937D9387
:1036A0008D939C9398970E94882388E080932805A7
:1036B0000DC01092F7011092F6010E94FE21909128
:1036C000F0018091F201981709F0E6C9E9960FB66A
:1036D000F894DEBF0FBECDBFCF91DF911F910F9148
:1036E000FF90EF90DF90CF90BF90AF909F908F9022
:1036F0007F906F905F904F903F902F900895FF9232
:103700000F931F93CF93DF931092F3011092F40164
:10371000C0E0D0E00C2FFC2E8091AA0690E00C2E89
:1037200002C0959587950A94E2F780FF08C0109132
:10373000F3018C2F0E94F31E182B1093F30180913C
:10374000AB0690E002C095958795FA94E2F780FF6A
:1037500008C01091F401802F0E94FD1E182B1093B9
:10376000F4012196C330D105A9F6DF91CF911F91C5
:103770000F91FF90089580916F008D7F80936F006F
:1037800080918100887F8160809381001092F50193
:103790009091AC069F3F21F48091290585FF0AC0D6
:1037A00080912805843031F0892F90E00E947227A3
:1037B00091E001C090E08091B60682FF02C081E0F6
:1037C0009827992311F0289A0895289808950E941F
:1037D000BB1B8BE2EAEFF1E0DF011D928A95E9F76E
:1037E00083E2EDECF1E0DF011D928A95E9F710929A
:1037F000EF011092EE011092F7011092F601109273
:10380000F0011092F10181E08093F2011092F50134
:103810000E947F1B8BB1837E9091F301892B8BB922
:103820008BB18F719091F401892B8BB908951F9200
:103830000F920FB60F9211242F933F934F935F93E4
:103840006F937F938F939F93AF93BF93CF93DF93A8
:10385000EF93FF938091F501882309F007C29BB194
:103860008091DC01807E9F71892B8BB98BB1837E27
:103870009091DB01892B8BB98091DA0186BD82E0C2
:1038800085BD81E08093F50178948091EE0190915F
:10389000EF01892B09F0A2C09091F0018091F10114
:1038A000891709F490C09091F00186E0989FE0019B
:1038B0001124C755DE4FD093EF01C093EE018B81E9
:1038C0009C8190938900809388008881998190934E
:1038D000EA018093E9019A818091EB01891761F1F6
:1038E0009093EB01E1E19E9FF0011124EC5AFE4F11
:1038F000F093ED01E093EC0185859685A785B0896D
:10390000B695A795979587958093CD019093CE0115
:10391000A093CF01B093D0018093D1019093D201B5
:10392000A093D301B093D4018093D5019093D60195
:10393000A093D701B093D801E091EC01F091ED0193
:103940008091F401908189278093DC012D81818110
:103950009281A381B481022E04C0B695A795979554
:1039600087950A94D2F78093DD019093DE01A093AE
:10397000DF01B093E00185819681A781B085022E99
:1039800004C0B695A795979587950A94D2F780932A
:10399000E1019093E201A093E301B093E4018185FA
:1039A0009285A385B48504C0B695A795979587950C
:1039B0002A95D2F78093E5019093E601A093E70161
:1039C000B093E8010BC00E94BB1B9FB7F894809195
:1039D00029058460809329059FBF48C10E94EE2B72
:1039E0001092DB012091DD013091DE014091DF0179
:1039F0005091E0018091CD019091CE01A091CF0135
:103A0000B091D001280F391F4A1F5B1F2093CD01B1
:103A10003093CE014093CF015093D001E091EC015F
:103A2000F091ED0185859685A785B089821793076A
:103A3000A407B507A8F584E08093DB01858596850A
:103A4000A785B089281B390B4A0B5B0B2093CD014E
:103A50003093CE014093CF015093D001808185FFF8
:103A60000CC080912B0590912C05A0912D05B09153
:103A70002E050197A109B1090BC080912B059091EA
:103A80002C05A0912D05B0912E050196A11DB11D0B
:103A900080932B0590932C05A0932D05B0932E05B4
:103AA0002091E1013091E2014091E3015091E40164
:103AB0008091D1019091D201A091D301B091D40114
:103AC000280F391F4A1F5B1F2093D1013093D20169
:103AD0004093D3015093D40185859685A785B089FD
:103AE00082179307A407B507B8F58091DB018860BA
:103AF0008093DB0185859685A785B089281B390BC6
:103B00004A0B5B0B2093D1013093D2014093D30138
:103B10005093D401808186FF0CC080912F05909135
:103B20003005A0913105B09132050197A109B10985
:103B30000BC080912F0590913005A0913105B09177
:103B400032050196A11DB11D80932F05909330057C
:103B5000A0933105B09332052091E5013091E60143
:103B60004091E7015091E8018091D5019091D601F3
:103B7000A091D701B091D801280F391F4A1F5B1FB0
:103B80002093D5013093D6014093D7015093D801AB
:103B900085859685A785B08982179307A407B50701
:103BA000B8F58091DB0180618093DB018585968586
:103BB000A785B089281B390B4A0B5B0B2093D501D5
:103BC0003093D6014093D7015093D801808187FF6D
:103BD0000CC08091330590913405A0913505B091CA
:103BE00036050197A109B1090BC080913305909169
:103BF0003405A0913505B09136050196A11DB11D82
:103C00008093330590933405A0933505B093360522
:103C100080912805843039F480912A059091DB0148
:103C200089238093DB018091E9019091EA0101975A
:103C30009093EA018093E901892B79F41092EF01C6
:103C40001092EE018091F0018F5F8093F0018091DE
:103C5000F001863011F41092F0018091F3019091FF
:103C6000DB0189278093DB011092F501FF91EF9131
:103C7000DF91CF91BF91AF919F918F917F916F9184
:103C80005F914F913F912F910F900FBE0F901F901A
:103C90001895F999FECF92BD81BD81E08FBB80B5AB
:103CA0000895F894F999FECF92BD81BD81E08FBB54
:103CB00040B54627842F992787FD9095262F30E021
:103CC00082239323892B39F06F3F19F060BD84E084
:103CD00006C084E104C0442321F060BD84E28FBBB0
:103CE000F99A789408958F929F92AF92BF92CF9253
:103CF000DF92EF92FF920F93DF93CF9300D0CDB777
:103D0000DEB75C016B017A014A0100E01EC00023AE
:103D100019F021E030E008C0202F332727FD30952F
:103D20002227330F221F3327F60161916F01062FDF
:103D3000020F9C012F5F3F4F3A8329830E94511E3F
:103D400008948108910889819A8181149104F9F677
:103D5000C7018A0D9B1D602F0E94511E0F900F906E
:103D6000CF91DF910F91FF90EF90DF90CF90BF90B8
:103D7000AF909F908F900895CF93DF93EC01FB015C
:103D80009A0190E0B1E019C0F999FECFF2BDE1BD12
:103D9000BFBBA0B5992319F081E090E008C0892F3E
:103DA000992787FD90958827990F881F9927319625
:103DB0009A2F980FA993215030402115310521F7F2
:103DC000460F571FF999FECF52BD41BD81E08FBB11
:103DD00080B520E030E0981711F421E030E0C9010F
:103DE000DF91CF910895882311F484E00895813004
:103DF00011F080E1089588E00895882311F480E2AD
:103E00000895813011F080E8089580E408958823B2
:103E100011F482E00895813011F088E0089584E083
:103E2000089580E090E00E94491E853011F020E066
:103E30000CC089E796E061E070E04DE450E00E943C
:103E4000BC1E20E0892B09F021E0822F089580E03C
:103E500093E060E00E94511E81E593E060E00E94E3
:103E6000511E089580E090E065E00E94511E81E0BF
:103E700090E069E776E04DE450E00E94731E0895FB
:103E8000CF92DF92EF92FF920F931F93082F6A0158
:103E90007B01CB01BA0120E030E040E050E00E941D
:103EA000CD33882314F484E017C1043608F459C0D4
:103EB000045690E0033008F04BC0913089F0913007
:103EC00030F09230D1F0933009F001C131C0E02FD1
:103ED000F0E0EE0FFF1FEE0FFF1FE758F94F08C08D
:103EE000E02FF0E0EE0FFF1FEE0FFF1FEB57F94F33
:103EF000C082D182E282F382EAC010E0000F111F7B
:103F0000000F111F0F56194FC701B60120E030E016
:103F100040E752E40E94163620E030E040E752E4E9
:103F20000E941636F8016083718382839383CFC029
:103F3000E02FF0E0EE0FFF1FEE0FFF1FE356F94FEB
:103F4000D701C601B05880839183A283B383BFC0D9
:103F50000A3008F4C0C09F5F943009F4BCC00A5016
:103F6000A9CFC701B6010E94F0360E944134E02F6C
:103F7000F0E0EC31F10508F0AEC0EC5CFF4FEE0F65
:103F8000FF1F0590F491E02D0994633010F486E052
:103F9000A3C06093A9069BC06093AC0698C06093D1
:103FA000AA0602C06093AB060E947F1B90C06623E6
:103FB00021F08091B606846009C08091B6068B7F9F
:103FC00005C0662331F08091B60680648093B60602
:103FD0007EC08091B6068F7BF9CF662321F0809159
:103FE000B6068068F3CF8091B6068F77EFCF6093E7
:103FF000AD06C092AE06D092AF06E092B006F09247
:10400000B10665C0C092B206D092B306E092B40683
:10401000F092B5065CC0662321F08091B6068160FF
:10402000D5CF8091B6068E7FD1CF662321F08091C7
:10403000B6068260CBCF8091B6068D7FC7CF662350
:1040400041F08091B60684FD02C08AE045C08062DE
:10405000BDCF8091B6068F7DB9CF662321F08091C8
:10406000B606886003C08091B606877F8093B60647
:104070000E94A5272CC0662321F08091B60680619E
:10408000A5CF8091B6068F7CA1CF6093B7061FC0E5
:10409000C092B806D092B906E092BA06F092BB067A
:1040A00016C0C092BC06D092BD06E092BE06F09249
:1040B000BF060DC06093C0061092C10608C0C09232
:1040C000C206D092C306E092C406F092C5060E94D2
:1040D000321F80E001C083E01F910F91FF90EF90AD
:1040E000DF90CF9008952AE02093A90688EC809372
:1040F000AC061092AA061092AB0683E08093AD0640
:104100008DEC9CECACE4BDE38093AE069093AF06DF
:10411000A093B006B093B1068FE692E1A3E0BBE3B3
:104120008093B2069093B306A093B406B093B506FD
:104130001092B70680E090E0A8ECB2E48093B80655
:104140009093B906A093BA06B093BB0680E090E0C6
:10415000A8E4B3E48093BC069093BD06A093BE068A
:10416000B093BF068AEF90E09093C1068093C0069B
:1041700080E090E0A0EAB0E48093C2069093C3068A
:10418000A093C406B093C5062093B60680E090E0E5
:10419000AAEFB4E48093790690937A06A0937B0605
:1041A000B0937C0680937D0690937E06A0937F0655
:1041B000B09380068093810690938206A093830635
:1041C000B093840680E090E0AAEFB3E48093850684
:1041D00090938606A0938706B093880680938906FD
:1041E00090938A06A0938B06B0938C0680938D06DD
:1041F00090938E06A0938F06B093900680E090EA8D
:10420000ACE0B7E48093910690939206A093930656
:10421000B09394068093950690939606A093970684
:10422000B09398068093990690939A06A0939B0664
:10423000B0939C0680E090E0A8ECB2EC80939D06E1
:1042400090939E06A0939F06B093A0068093A1062C
:104250009093A206A093A306B093A40680E090E0FA
:10426000A8E4B3EC8093A5069093A606A093A706B6
:10427000B093A8060E94321F08959DE0899FC00157
:10428000112480509E4F4CE050E00E94731E089510
:104290000F931F93CF93DF93162F072F9DE0899FD6
:1042A000E0011124C050DE4F862F972FBE014CE055
:1042B00050E00E94BC1E892B11F081E00FC0E12F5D
:1042C000F02F8CE0DF011D928A95E9F7CE01612F76
:1042D000702F4CE050E00E94731E80E0DF91CF9180
:1042E0001F910F910895EF92FF921F93DF93CF9349
:1042F000CDB7DEB72C970FB6F894DEBF0FBECDBF9B
:104300000E94111F882371F487E00E94722C0E9482
:1043100073200E94271F8EEA93E060E00E94511EE6
:104320000E946F2F10E07E010894E11CF11C812F88
:10433000B7010E944821882319F487E00E94722C5B
:104340001F5F1830A1F72C960FB6F894DEBF0FBE92
:10435000CDBFCF91DF911F91FF90EF900895BC01E9
:104360008EEA93E040E550E00E94731E0895CF93DB
:10437000DF93EC016EEA73E040E550E00E94BC1E62
:10438000892B11F081E009C018828EEA93E0BE010A
:1043900040E550E00E94731E80E0DF91CF910895C8
:1043A00091E5899FC001112480509D4F40E550E068
:1043B0000E94731E08950F931F93CF93DF938B0179
:1043C00091E5899FE0011124C050DD4FCB01BE0172
:1043D00040E550E00E94BC1E892B11F081E009C02D
:1043E000F8011082CE01B80140E550E00E94731E32
:1043F00080E0DF91CF911F910F91089520910705E3
:1044000080910805821769F0922F9F5F923109F41D
:1044100090E080910A05281711F490930A05909373
:10442000070508959091070580910805891719F4EB
:1044300020E030E006C089E2989F900111242B5DB6
:104440003D4FC901089520E090910705809109052D
:10445000981709F421E0822F089580912B059091FF
:104460002C05A0912D05B0912E0580930B059093FE
:104470000C05A0930D05B0930E0580912F0590912A
:104480003005A0913105B091320580930F059093CE
:104490001005A0931105B0931205809133059091FA
:1044A0003405A0913505B09136058093130590939E
:1044B0001405A0931505B09316050895809108057D
:1044C00090910705891710F0891B08958E5E891B4E
:1044D00008954F925F926F927F928F929F92AF92C8
:1044E000BF92CF92DF92EF92FF920F931F93CF93E1
:1044F000DF9380910805882309F482E1782E7A946D
:1045000060900A05761409F4F2C089E2789E4001B1
:10451000112485E292E0880E991EF401A588B688E0
:10452000C788D08C21A132A143A154A1CA01B901ED
:104530000E94F432F40125A136A147A150A50E94A2
:1045400016367B018C01B501C601A80197010E94B6
:10455000CD3387FD04C0D801C70157016D01C501E6
:10456000D601F401818B928BA38BB48B772011F44D
:1045700032E1732E7A94761409F04EC080910705CB
:10458000681609F050C00E940F154DC0769CE001DE
:104590001124CB5DDD4F772011F422E1722E7A9445
:1045A00080910705781611F40E940F15AD88BE881A
:1045B000CF88D88C69897A898B899C89A6019501D5
:1045C0000E94CD33882331F129A13AA14BA15CA1EE
:1045D000CA01B9010E94F4322DA13EA14FA158A5F4
:1045E0000E941636F40121893289438954890E9438
:1045F000F4327B018C01A60195010E94CD33882302
:104600002CF4E98AFA8A0B8B1C8B04C0A98ABA8A1B
:10461000CB8ADC8A4E0102C099E2692E80910A059C
:10462000781609F0B3CFA0900A05BA2CB394F2E142
:10463000BF1609F4BB2489E2A89E800111240B5DFA
:104640001D4F5090080589E2482E4CC0B49CE001F3
:104650001124CB5DDD4FF801C188D288E388F4884E
:1046600069887A888B889C88C701B601A401930168
:104670000E94CD3388231CF5F80121A132A143A16A
:1046800054A1CA01B9010E94F432F80125A136A152
:1046900047A150A50E9416369B01AC01C701B60187
:1046A0000E94F4327B018C01A40193010E94CD335E
:1046B00088232CF4E98AFA8A0B8B1C8BAB2C698932
:1046C0007A898B899C892D893E894F89588D0E94D2
:1046D000CD33882309F4AB2CB394F2E1BF1609F46F
:1046E000BB248E01B51409F0B1CFA0920A05DF9169
:1046F000CF911F910F91FF90EF90DF90CF90BF90DF
:10470000AF909F908F907F906F905F904F900895A3
:104710000E940F158091070580930A050E94692267
:104720000895209107052F5F223109F420E0809140
:104730000805281729F460E070E080E090E012C0DE
:1047400030E089E290E0289FF001299FF00D389F2A
:10475000F00D1124EB5DFD4F618972898389948985
:104760000E94A33608952F923F924F925F926F92CC
:104770007F928F929F92AF92BF92CF92DF92EF92F1
:10478000FF920F931F93DF93CF93CDB7DEB7E097E0
:104790000FB6F894DEBF0FBECDBF98A78FA349A771
:1047A0005AA76BA77CA7222E9091080589E2989FB3
:1047B0004001112425E232E0820E931ED4011D96A1
:1047C0001D921D921D921C92509780E090E0A0E0F7
:1047D000B0E0F40185A396A3A7A3B0A7108289E94E
:1047E00096E7A6E9BEE781A392A3A3A3B4A32401FD
:1047F000332466247724F301E758F94FA080B18071
:10480000C280D380EFA1F8A5E60DF71DC601B50162
:1048100020813181428153810E9416360E94E63503
:104820009B01AC01E1E0F0E0EC0FFD1FE60DF71D90
:104830002083318342835383F301E55FFA4F808104
:104840009181A281B381281B390B4A0B5B0BDA01E2
:10485000C90157FF07C088279927DC01821B930BEA
:10486000A40BB50BF20181839283A383B483F4017B
:10487000E584F684078510898E159F05A007B1078A
:1048800010F4D801C701F40185879687A787B08BFC
:10489000CA01B9010E946F34A60195010E94D43368
:1048A0005B016C01EDE0F0E0EC0FFD1FE60DF71D84
:1048B000608371838283938320E030E040E050E0A6
:1048C0000E94CD33882344F4D4011C91832D0E948F
:1048D000FD1E182BF4011083D4019596ED90FD90E8
:1048E0000D911C919897C601B501A60195010E94F2
:1048F00016369B01AC01C801B7010E94F4327B015E
:104900008C01CB01D801F40185A396A3A7A3B0A77E
:10491000339424E030E0620E731E420E531E33E0E7
:10492000331609F068CFB701C8010E94A3367B0196
:104930008C01D40195966D937D938D939C9398975C
:104940001D968D919D910D90BC91A02D0097A10574
:10495000B10509F4E5C169A57AA58BA59CA520E060
:1049600030E040E050E00E94CD3388232CF489E908
:1049700096E7A6E9BEE71EC0222061F0C801B70194
:1049800029A53AA54BA55CA50E94D43369A77AA7AF
:104990008BA79CA769A57AA58BA59CA520E030E0F4
:1049A00040E85FE30E94CD33882344F480E090E048
:1049B000A0E8BFE389A79AA7ABA7BCA760E070E017
:1049C00080E89FE3A80197010E94D4336BA37CA3E6
:1049D0008DA39EA3DE011D96BE8FAD8FE7E1F5E0AE
:1049E000FC8FEB8F25E836E03A8F298F80E090E04E
:1049F000A0E0B0E08F8F98A3A9A3BAA3DE015996D7
:104A0000B8ABAFA7ED8DFE8DE080F1800281138100
:104A1000C801B70120E030E040E050E00E94CD3313
:104A2000882309F47CC0C801B7012BA13CA14DA18A
:104A30005EA10E9416362B013C01AD8DBE8D6D939B
:104A40007D938D939C93139760E070E080E89FE3E3
:104A5000A30192010E94D4335B016C01E894D7F862
:104A6000C601B501E98DFA8D2081318142815381E2
:104A70000E9416367B018C0169A57AA58BA59CA5A1
:104A8000A80197010E94CD3387FD04C0E9A6FAA6CC
:104A90000BA71CA7D4019196BC91BDA7F401F2A16C
:104AA000FEA7D40193962C90939794963C90C601C0
:104AB000B501E98DFA8D24853585468557850E9497
:104AC00016367B018C016DA57EA5C101A801970159
:104AD0000E94CD3387FD05C0D801C701EDA69EA772
:104AE0001D018DA59EA5D101F40181A392A3A3A3CD
:104AF000B4A3C301B201AB8DBC8D2D913D914D91FD
:104B00005C910E9416369B01AC016F8D78A189A142
:104B10009AA10E94F3326F8F78A389A39AA3ED8D97
:104B2000FE8D3496FE8FED8F2B8D3C8D2C5F3F4F8D
:104B30003C8F2B8F898D9A8D04969A8F898FAFA584
:104B4000B8A9EA17FB0709F05DCF9091080580919D
:104B50000705981771F480E090E0A0E0B0E0F40160
:104B6000818B928BA38BB48B818F928FA38FB48F09
:104B700052C060E070E080E89FE32F8D38A149A12A
:104B80005AA10E94F33220E030E040E05FE30E944F
:104B900016360E94A3365B016C01D40191966D918B
:104BA0007D918D919C9194972091AE063091AF06A6
:104BB0004091B0065091B1060E941636A6019501AB
:104BC0000E9416367B018C0160E070E080E89FE374
:104BD000A60195010E94F3329B01AC01C801B70107
:104BE0000E94D4337B018C0120E030E040E050E0B3
:104BF0000E94CD33882354F40F2EF0E0EF2EF0E026
:104C0000FF2EF0E00F2FF0E01F2FF02DF401E18ECA
:104C1000F28E038F148F69A57AA58BA59CA59B01A5
:104C2000AC010E9416367B018C01D4015D966D9318
:104C30007D938D939C93909759965C9059975A9633
:104C40004C905A975B963C905B975C962C90D090DA
:104C50002305C0902405B0902505A09026052D2D94
:104C60003C2D4B2D5A2D0E94CD3387FD04C06D2C59
:104C70007C2CF50105C0D801C7013701FA2FEB2FB5
:104C8000652D742D832D922D93014F2F5E2F0E9441
:104C9000CD3388232CF4852D942DA32DB22D0EC059
:104CA000C801B7012D2D3C2D4B2D5A2D0E94CD331F
:104CB00087FD06C08D2D9C2DAB2DBA2D7C018D015D
:104CC000F401E58AF68A078B108FA7E1B5E0FE01B3
:104CD0003D968CE001900D928150E1F7F401858DB5
:104CE000968DA78DB0A18093230590932405A09362
:104CF0002505B0932605ABE0B5E0FE0131968CE0CA
:104D000001900D928150E1F780910905809308058B
:104D10008F5F823109F480E0809309050E94692247
:104D2000E0960FB6F894DEBF0FBECDBFCF91DF91F6
:104D30001F910F91FF90EF90DF90CF90BF90AF90B9
:104D40009F908F907F906F905F904F903F902F90AB
:104D500008958CE1EBE0F5E0DF011D928A95E9F71B
:104D6000109207051092080581E0809309051092C2
:104D70000A0508956F927F928F929F92AF92BF9291
:104D8000CF92DF92EF92FF920F931F93CF93DF9317
:104D90004C013B015A01FB018081F401E80FF11D38
:104DA000EF0189918D3229F481812196CC24C3941D
:104DB00005C08B3211F481812196CC2420E030E0B3
:104DC00040E050E0DD24E0E070E0682F60536A309E
:104DD000F8F4EF5FE930C0F47111DA94DA01C90137
:104DE000F2E0880F991FAA1FBB1FFA95D1F7280F71
:104DF000391F4A1F5B1F220F331F441F551F260FE9
:104E0000311D411D511D09C0772339F4D39405C0CC
:104E10006E3F29F4772319F471E08991D6CFEE2300
:104E200011F480E050C0CA01B9010E946D347B01C9
:104E30008C0120E030E040E050E00E94CD33882338
:104E400069F42BC0C801B7012AE037ED43E25CE307
:104E50000E9416367B018C01F2E0DF0E8FEFD81630
:104E60008CF3D81659F4C801B7012DEC3CEC4CEC8E
:104E70005DE30E9416367B018C010FC0DD2069F0D6
:104E8000C801B70120E030E040E251E40E9416364C
:104E90007B018C01DA941D149CF3CC2049F0D801DD
:104EA000C701B058F50180839183A283B38305C005
:104EB000F501E082F18202831383882D80958C0FA7
:104EC000F301808381E0DF91CF911F910F91FF90DB
:104ED000EF90DF90CF90BF90AF909F908F907F909A
:104EE0006F90089520EA3FE004C0F9013197F1F78F
:104EF00001970097D1F70895AF92BF92CF92DF92BA
:104F0000EF92FF920F931F937B018C0159016A016D
:104F1000A80197010E9416367B018C01C601B501DC
:104F2000A60195010E9416369B01AC01C801B7018C
:104F30000E94F4320E94A3361F910F91FF90EF90D0
:104F4000DF90CF90BF90AF90089584B1817F84B9F6
:104F50008091B606982F86FF03C085B1817F02C07D
:104F600085B18E6085B993FF09C080916B008E601A
:104F700080936B0080916800816008C080916B0015
:104F8000817F80936B00809168008E7F80936800A2
:104F90000895EBE6F0E08081817F8083E8E6F0E031
:104FA00080818E7F80830895CF92DF92EF92FF926F
:104FB0000F931F93CF93DF936C01C0E0D0E0F60115
:104FC000EC0FFD1FE080F18002811381C801B70161
:104FD00020E030E040E050E00E94DB3518166CF035
:104FE000FE01E758F94FC801B70124A135A146A138
:104FF00057A10E94CD33882304F580912805803184
:1050000079F49FB7F89480912905886080932905E9
:105010009FBF0E947613809127058823D1F312C089
:105020000E942D049FB7F894809129058066809393
:1050300029059FBF0E94761305C02496CC30D10568
:1050400009F0BDCFDF91CF911F910F91FF90EF90AD
:10505000DF90CF9008951F920F920FB60F921124F8
:105060002F933F934F935F936F937F938F939F9370
:10507000AF93BF93EF93FF9380912805813071F038
:105080008091290585FD0AC00E942D049FB7F894E0
:10509000809129058066809329059FBFFF91EF913C
:1050A000BF91AF919F918F917F916F915F914F9140
:1050B0003F912F910F900FBE0F901F9018952F9238
:1050C0003F924F925F926F927F928F929F92AF9298
:1050D000BF92CF92DF92EF92FF920F931F93DF93D5
:1050E000CF93CDB7DEB7A3970FB6F894DEBF0FBE50
:1050F000CDBF8F8F80912705882309F0E2C1809171
:10510000BC069091BD06A091BE06B091BF068F8BE4
:10511000988FA98FBA8F4DE9A42E46E0B42E66244D
:10512000772488249924CC24DD241E010894211C92
:10513000311C34E0432E512C4C0E5D1E8C2D0E94F0
:10514000071FF101EC0DFD1D80838C2D0E94F31EC5
:10515000F201EC0DFD1D8083D501ED90FD900D91C8
:105160001C91B301C401A80197010E94DB351816F8
:1051700024F0C301D4017C018D010894C11CD11C11
:10518000E4E0F0E0AE0EBF1EF3E0CF16D10429F04C
:10519000D801C70137014D01D1CFC801B70120E0C7
:1051A00030E040EC5FEB0E9416365B016C010E9420
:1051B000A92601E023E02D8B27E0422E512C4C0E36
:1051C0005D1E9F8D892F90E099A388A3350146012C
:1051D00097FA909497F890948091B60686FD02C055
:1051E0000E8B03C0A1E0A027AE8B8091B706E82EFE
:1051F000FF241201920160E010E040E050E0742FC3
:1052000088A199A1042E02C0959587950A94E2F78A
:10521000FC01E170F070FBA3EAA380FF10C06F5F98
:10522000002339F4D9016D927D928D929C9213974F
:105230000FC0F901A082B182C282D38209C080E08E
:1052400090E0A0E0B0E0F90180839183A283B38372
:10525000C70102C0959587957A95E2F780FF0AC04D
:10526000F90180819181A281B381B05880839183BB
:10527000A283B3838AA19BA1892B41F0E4E0F0E0F3
:10528000EC0FFD1FE40FF51F8081182B4F5F5F4F60
:105290002C5F3F4F4330510509F0B1CF70E080E003
:1052A00090E00E946D340E94A3369B01AC011093E4
:1052B0002A056F89788D898D9A8D0E941636AB01EB
:1052C000BC01C20120E00E94B3230E9431150E945C
:1052D000AF1443B19E89992311F0AEE04A2720E034
:1052E00030E0E4E0F0E0EC0FFD1FE20FF31F9081EF
:1052F000812F892359F0E1E0F0E0EC0FFD1FE20F70
:10530000F31F8081842311F0909519232F5F3F4F65
:105310002330310531F710932A050E943115809111
:10532000290584FF03C00E947613CBC0812F8C71A6
:1053300081F60E94E71B0E94A9268091C0069091E9
:10534000C1060E9472278091B8069091B906A0917B
:10535000BA06B091BB068F8B988FA98FBA8F9D89A3
:10536000992329F0A1E00A2791509D8B35CF809198
:10537000B706E82FF0E0FC8BEB8B4090C206509014
:10538000C3066090C4067090C506D301C201B05830
:105390008B8F9C8FAD8FBE8F9BE2C92E95E0D92E4F
:1053A00089E7A82E86E0B82E8824992488A199A19F
:1053B000082C02C0959587950A94E2F780FF3DC0BE
:1053C0008B899C89082C02C0959587950A94E2F7F1
:1053D00080FF23C0D5019496ED90FD900D911C9116
:1053E0009797C301B201A80197010E94F432F1011D
:1053F0006083718382839383C801B701D5012D91A6
:105400003D914D915C910E9416360E94E635F60161
:10541000608371838283938323C08B8D9C8DAD8D3C
:10542000BE8DF10180839183A283B383D6011D9247
:105430001D921D921C92139713C0F6016081718119
:10544000828193810E946F34D5012D913D914D91C0
:105450005C910E94D433F1016083718382839383D2
:105460000894811C911C24E030E0220E331EC20EF1
:10547000D31EA20EB31E33E08316910409F096CF1B
:105480000E942D224091BC065091BD066091BE063F
:105490007091BF06CE01079620E00E94B32388E0FA
:1054A000809328059FB7F8948091290582608093A6
:1054B00029059FBF0E9476130E94101484E08093F8
:1054C0002805A3960FB6F894DEBF0FBECDBFCF91CF
:1054D000DF911F910F91FF90EF90DF90CF90BF90E1
:1054E000AF909F908F907F906F905F904F903F9084
:1054F0002F9008958F929F92AF92BF92CF92DF929A
:10550000EF92FF920F931F93DF93CF93CDB7DEB748
:105510002A970FB6F894DEBF0FBECDBF7B018C017A
:10552000A42E20E030E040E050E00E94CD338823FC
:105530003CF48DE20E94AE1217FB109517F91095FE
:10554000DA2C0CC0C801B70120E030E048EC52E48E
:105550000E9416367B018C018EEFD80EE1E0ED152E
:1055600088F3A0FE0AC0C801B70120E030E040E2A5
:1055700051E40E9416367B018C01C801B70120E07E
:1055800030E040E05FE30E94F4320E943C346B0163
:105590007C019E012F5F3F4FF901EA0DF11D8EE264
:1055A0008083BB2449011EC0BA1409F4B39484015A
:1055B0000B0D111DC701B6012AE030E040E050E0BC
:1055C0000E941B37605DF8016083B394C701B60188
:1055D0002AE030E040E050E00E941B37C901DA01C8
:1055E0006C017D01C114D104E104F104E9F606C0A7
:1055F000FC01EB0DF11D2083B39403C0CE01019695
:1056000020E3BA14A8F3BA1489F48B2D8F5FFE013E
:10561000E80FF11D90E39183B82EB39407C0FE010B
:10562000EB0DF11D80810E94AE12BA94BB20B9F738
:105630002A960FB6F894DEBF0FBECDBFCF91DF9193
:105640001F910F91FF90EF90DF90CF90BF90AF90A0
:105650009F908F90089543E00E947A2A08959B01BD
:10566000AC018091B60680FF0AC0CA01B9012BE8DF
:1056700032E441E25DE30E94163641E003C0CA0114
:10568000B90140E00E947A2A08959B01AC01809103
:10569000B60680FF0AC0CA01B9012BE832E441E234
:1056A0005DE30E94163644E003C0CA01B90143E03D
:1056B0000E947A2A08951F93DF93CF9300D00F9210
:1056C000CDB7DEB7282F882321F480E30E94AE12E5
:1056D0001EC010E0AE014F5F5F4FFA01E10FF11DF8
:1056E000822F6AE00E940F37905D90831F5F822FA8
:1056F0000E940F37282F882381F707C0FE01E10F92
:10570000F11D80810E94AE1211501123B9F70F9044
:105710000F900F90CF91DF911F9108950F931F93DA
:10572000DF93CF93CDB7DEB728970FB6F894DEBFDF
:105730000FBECDBF982FFE0131969E01275F3F4FD0
:10574000892F817081939695E217F307C9F78E012F
:10575000085F1F4FF8018081805D0E94AE120150EA
:1057600010400C171D07B1F728960FB6F894DEBF4E
:105770000FBECDBFCF91DF911F910F910895CF93B1
:10578000DF93EC0102C00E94AE12FE0121968491CB
:105790008823C9F7DF91CF910895CF93DF93EC0170
:1057A00003C021960E94AE1288818823D1F7DF9131
:1057B000CF9108953D988091B60687FF04C0459823
:1057C0001092C6060895459A80E28093C606089511
:1057D00086B180729091C606892708958091380518
:1057E0008130B1F486B180729091C606891781F03C
:1057F00010923805E9E3F5E0DF011E978CE00D908B
:1058000001928150E1F780912905886080932905F4
:1058100008958DE994E00E94BF2B089581EE95E0F4
:105820000E94BF2B08951F93182F83E596E00E94D6
:10583000BF2B133091F0143028F4113041F01230A6
:10584000B1F408C0143061F0153089F40CC081E463
:1058500096E00BC08DE296E008C08BE196E005C0B3
:1058600083E196E002C08AE096E00E94BF2B86E0CA
:1058700096E00E94BF2B1F910895FF920F931F93F4
:10588000CF93DF9388EF91E00E94BF2B09E315E0EF
:10589000C9E7D6E0FF24F80160817181828193819C
:1058A0000E946F34288139814A815B810E94D43300
:1058B0000E94452BF2E0FF1621F086EF91E00E9456
:1058C000BF2BF3940C5F1F4F249683E0F81619F753
:1058D00082EF91E00E94BF2BDF91CF911F910F913A
:1058E000FF9008951F93182F882319F485EA97E0F5
:1058F0005CC08DE997E00E94BF2B1730A9F11830EA
:1059000078F4133029F1143030F41130C9F012302A
:1059100009F042C018C0153009F1163010F51BC04F
:105920001B3071F11C3028F4193021F11A3028F5A0
:105930001EC0153141F1163161F1143169F526C0EF
:1059400085E897E002C083E797E00E94BF2B2BC059
:1059500081E697E0FACF87E597E0F7CF86E497E016
:10596000F4CF87E397E0F1CF86E197E0EECF8DE0CB
:1059700097E0EBCF82E097E0E8CF8FEE96E0E5CFBF
:1059800081EE96E0E2CF8BEC96E0DFCF87EB96E0FE
:10599000DCCF83EA96E0D9CF81E996E00E94BF2B65
:1059A000812F0E945B2B8EE896E00E94BF2B1F91F7
:1059B0000895DF92EF92FF920F931F93DF93CF939F
:1059C000CDB7DEB768970FB6F894DEBF0FBECDBF78
:1059D000DE011196EBE2F5E08CE001900D92815032
:1059E000E1F7809128058430E1F0853038F481308A
:1059F000D9F0813050F08230F1F419C0803159F083
:105A0000803261F08830B9F403C082E391E011C0C4
:105A10008BE291E00EC086E291E00BC080E291E063
:105A200008C08AE191E005C083E191E002C08CE00A
:105A300091E00E94BF2B8091AD06082F10E0C801B5
:105A400083709070892BE1F169817A818B819C81CF
:105A50000E946F342091790630917A0640917B063E
:105A600050917C060E94D4336D877E878F87988BF8
:105A70006D817E818F8198850E946F3420917D0693
:105A800030917E0640917F06509180060E94D4336B
:105A9000698B7A8B8B8B9C8B69857A858B859C85B2
:105AA0000E946F34209181063091820640918306D6
:105AB000509184060E94D4336D8B7E8B8F8B988F90
:105AC00000FF1EC085E091E00E94BF2B6D857E85A2
:105AD0008F8598890E94452B83E091E00E94BF2B1F
:105AE00069897A898B899C890E94452B83E091E0A2
:105AF0000E94BF2B6D897E898F89988D0E94452BCE
:105B00008091AD0681FF50C08CEF90E00E94BF2BCA
:105B10008E01035F1F4F84E6E82E85E0F82EDD241A
:105B2000F701608171818281938124853585468565
:105B300057850E94F4329B01AC01F80160817181AC
:105B4000828193810E94F332F801608371838283A2
:105B50009383F2E0DF1679F420917C0530917D0586
:105B600040917E0550917F050E94F332F8016083D9
:105B7000718382839383F801608171818281938133
:105B80000E94452BF2E0DF1621F08AEF90E00E94A0
:105B9000BF2BD3940C5F1F4F84E090E0E80EF91EFA
:105BA00093E0D91609F0BCCF8091AD0682FF08C002
:105BB00084EF90E00E94BF2B0E945E220E945B2B2C
:105BC0008091AD0683FF08C08FEE90E00E94BF2B4E
:105BD0000E948D120E945B2B8BEE90E00E94BF2BE7
:105BE00068960FB6F894DEBF0FBECDBFCF91DF91A0
:105BF0001F910F91FF90EF90DF9008950F931F93E7
:105C00008C018CE391E00E94BF2BC8010E94CD2B38
:105C100088E391E00E94BF2B1F910F910895FF929E
:105C20000F931F93F82E8B0189E591E00E94BF2B03
:105C30008F2D0E945B2B87E591E00E94BF2BC8014E
:105C40000E94CD2B84E591E00E94BF2B1F910F9104
:105C5000FF90089580914505823091F0833028F4BB
:105C6000882341F08130B1F408C0833061F0853081
:105C700089F40CC087EC91E00BC083EC91E008C084
:105C80008FEB91E005C08BEB91E002C086EB91E0D9
:105C90000E94BF2B83EB91E00E94BF2B80914B05AC
:105CA0008A5C0E945B2B80914905813041F08130F4
:105CB00018F0823059F406C08EEA91E005C089EAF6
:105CC00091E002C084EA91E00E94BF2B80914705D9
:105CD000882319F48FE991E002C08AE991E00E94DB
:105CE000BF2B80914805882319F485E991E002C013
:105CF00080E991E00E94BF2B80914605813019F424
:105D00008BE891E002C086E891E00E94BF2B809171
:105D10004C05813041F0813018F0823059F406C0D2
:105D200082E891E005C08EE791E002C08AE791E049
:105D30000E94BF2B80914E05813029F0813048F0C0
:105D4000823059F403C086E791E005C082E791E014
:105D500002C08EE691E00E94BF2B80914D05882302
:105D600019F0823041F403C08AE691E002C086E671
:105D700091E00E94BF2B83E691E00E94BF2B8091AF
:105D800057050E945B2B80E691E00E94BF2B60913B
:105D900053057091540580915505909156050E94C8
:105DA0002F2B8CE591E00E94BF2B0895CF92DF92BC
:105DB000EF92FF920F931F93DF93CF93CDB7DEB790
:105DC0002C970FB6F894DEBF0FBECDBFEE246E0148
:105DD0000894C11CD11C8E2DB6010E944821882335
:105DE00021F487E00E94722C6BC08FEE91E00E943C
:105DF000BF2B86E0E81621F0E7E0EE1649F403C079
:105E00008CEE91E002C089EE91E00E94BF2B04C0AD
:105E10008E2D8A5C0E945B2B87EE91E00E94BF2B47
:105E20008601FF24F80160817181828193810E9443
:105E3000452BF2E0FF1619F085EE91E002C081EEED
:105E400091E00E94BF2BF3940C5F1F4F83E0F81684
:105E500049F7E394E8E0EE1609F0BDCF8BED91E051
:105E60000E94BF2B00E715E0FF24F80160817181DB
:105E7000828193810E94452BF2E0FF1619F089ED93
:105E800091E002C085ED91E00E94BF2BF3940C5F7E
:105E90001F4F83E0F81649F78FEC91E00E94BF2B6B
:105EA00060917C0570917D0580917E0590917F05C4
:105EB0000E94452B8BEC91E00E94BF2B0E943D2C51
:105EC0002C960FB6F894DEBF0FBECDBFCF91DF91F9
:105ED0001F910F91FF90EF90DF90CF900895FF9268
:105EE0000F931F93CF93DF9389E994E00E94BF2B18
:105EF0008091A9060E945B2B80E894E00E94BF2B52
:105F00008091AC060E945B2B82E694E00E94BF2B3E
:105F10008091AA060E945B2B89E494E00E94BF2B2B
:105F20008091AA060E948E2B82E494E00E94BF2BEF
:105F30008091AB060E945B2B8AE294E00E94BF2B0B
:105F40008091AB060E948E2B83E294E00E94BF2BCF
:105F50008091B60690E09695879596958795817085
:105F60000E945B2B82E094E00E94BF2B8091B606DA
:105F700090E066E0969587956A95E1F781700E94BA
:105F80005B2B82EE93E00E94BF2B90E08091B606DF
:105F900087FD91E0892F0E945B2B82EC93E00E94A9
:105FA000BF2B8091AD060E945B2B8CEA93E00E9490
:105FB000BF2B8091AD060E948E2B84EA93E00E9455
:105FC000BF2B6091AE067091AF068091B0069091A4
:105FD000B1060E942B2B84E893E00E94BF2B6091B6
:105FE000B2067091B3068091B4069091B5060E94F6
:105FF0002B2B89E693E00E94BF2B8091B60681701F
:106000000E945B2B8CE493E00E94BF2B8091B6062C
:1060100090E09695879581700E945B2B82E393E0D8
:106020000E94BF2B8091B60690E045E0969587953B
:106030004A95E1F781700E945B2B87E193E00E9413
:10604000BF2B8091B60690E033E0969587953A9500
:10605000E1F781700E945B2B8CEF92E00E94BF2BD6
:106060008091B60690E024E0969587952A95E1F711
:1060700081700E945B2B80EE92E00E94BF2B80918A
:10608000B7060E945B2B86EC92E00E94BF2B8091AA
:10609000B7060E948E2B8EEB92E00E94BF2B609180
:1060A000B8067091B9068091BA069091BB060E941D
:1060B0002B2B81EA92E00E94BF2B6091BC0670916D
:1060C000BD068091BE069091BF060E942B2B84E8EE
:1060D00092E00E94BF2B8091C0060E945B2B85E658
:1060E00092E00E94BF2B6091C2067091C30680911E
:1060F000C4069091C5060E942B2B8CE492E00E946E
:10610000BF2B10E094E6F92E6AC08AE492E00E9468
:10611000BF2B802F8F0D0E945B2B88E492E00E94A2
:10612000BF2B113061F0113028F0123069F01330BC
:10613000E9F415C0688179818A819B8115C06C85DD
:106140007D858E859F8510C0688D798D8A8D9B8D0C
:1061500020E030E041E655E40E94D43305C06CA154
:106160007DA18EA19FA190580E942B2B85E492E0E7
:106170000E94BF2B013041F0013018F0023059F479
:1061800006C083E492E005C081E492E002C08FE3A0
:1061900092E00E94BF2B113051F0113028F01230E4
:1061A00049F0133071F409C085E392E008C083E23E
:1061B00092E005C082E192E002C082E092E00E949B
:1061C000BF2B8EEF91E00E94BF2B0F5F2496033010
:1061D00009F09BCF1F5F143031F08AE0F80EC9E759
:1061E000D6E000E092CFDF91CF911F910F91FF9009
:1061F00008951F93182F86E896E00E94BF2B1E3F3C
:1062000041F01F3F19F01D3F59F406C086E796E0A4
:1062100005C083E696E002C088E596E00E94BF2BA9
:1062200085E596E00E94BF2B84EF91E00E947227E3
:106230001F91089587B1887F87B988B1876088B931
:10624000ECE6F0E0808187608083E8E6F0E0808122
:106250008260808308951F920F920FB60F921124CF
:106260002F933F934F935F936F937F938F939F935E
:10627000AF93BF93EF93FF9386B190E08095909595
:1062800087709070892B91F0309903C00E942D0483
:106290000DC0319904C080912905886005C03299EC
:1062A00005C080912905826080932905FF91EF91B7
:1062B000BF91AF919F918F917F916F915F914F911E
:1062C0003F912F910F900FBE0F901F901895CF9375
:1062D000DF93EC0180E0BE010E94DB21882351F0B6
:1062E0008881882351F0CE010E94CD2BCE010E94DF
:1062F000E20801C087E00E94722C81E0BE010E948A
:10630000DB21882311F487E009C08881882341F0CC
:10631000CE010E94CD2BCE010E94E2080E94722C79
:10632000DF91CF910895DF92EF92FF920F931F9329
:10633000DF93CF93CDB7DEB729970FB6F894DEBFC2
:106340000FBECDBF7C0181E08983F7018181873455
:1063500019F188345CF4833449F184340CF050C072
:10636000882341F0843209F04BC007C0883509F01A
:1063700047C034C00E94092C26C182E08983F701FE
:106380008281882309F019C180912805807309F062
:1063900016C10E946F2F17C182E08983F7018281A5
:1063A000882309F00AC10E942A2E0DC192E0998328
:1063B000F7018281882309F000C18091280582308D
:1063C00021F40E942D0485E006C0882309F0F7C05F
:1063D0009093280584E00E94132CF5C082E0898305
:1063E000F7018281882309F0E8C080912805813077
:1063F00009F0E9C083E00E94132C10922805E3C045
:1064000090912805923008F0DAC0893439F18A3445
:106410002CF4833241F0883421F40FC08E3409F417
:1064200043C0DD2468C082E08983F701828188232C
:1064300009F0C3C00E94D62EC6C08091B60684FD66
:1064400002C015E0C1C00E944C048091270588233A
:1064500009F0B9C0C7010E946731B5C082E08983E5
:10646000F7018281882339F4C7010E94B721C7014F
:106470000E94FE2DA8C08D3309F09FC083E0898360
:106480008981F701E80FF11D80813397808389812D
:10649000F701E80FF11D90818F5F8983992381F7C0
:1064A000C7010E94AF218FC082E08983F7018281FA
:1064B0008823E1F4B7010E94DB21882329F080E0E2
:1064C000B7010E940F2E03C087E00E94722C81E06A
:1064D000B7010E94DB21882321F487E00E94722CFF
:1064E00072C081E0B7010E940F2E6DC0992309F0A0
:1064F00066C0DD24D394C7018E010F5F1F4FB80122
:10650000AE014E5F5F4F0E94BA26882309F459C03E
:106510009981F701E90FF11D80818D3309F04DC09C
:10652000892F8F5F8983DD2041F1482F50E0298139
:10653000822F90E0FC01E41BF50BEE0DFF1DD7014F
:10654000A80FB91F8C9180838C912F5F298388239A
:1065500071F7C7010E94E208182F8823A9F56A8104
:106560007B818C819D810E94F0360E944134DC0148
:10657000CB01B7010E94D02127C0C701B801AE01ED
:106580004A5F5F4F0E94BA268823D9F08981E80EBE
:10659000F11CF7018081882381F46A817B818C81E1
:1065A0009D810E944134DC01CB014E815F81688571
:1065B00079850E94401F182F07C013E005C018E01E
:1065C00003C012E001C010E0812F29960FB6F894A5
:1065D000DEBF0FBECDBFCF91DF911F910F91FF9016
:1065E000EF90DF9008955058BB27AA270ED081C2A4
:1065F00041D230F046D220F031F49F3F11F41EF426
:1066000011C20EF4E095E7FBDCC1E92F94D280F3D0
:10661000BA17620773078407950718F071F49EF59F
:10662000C3C20EF4E0950B2EBA2FA02D0B01B901B9
:1066300090010C01CA01A0011124FF27591B99F0F8
:10664000593F50F4503E68F11A16F040A22F232F04
:10665000342F4427585FF3CF469537952795A79554
:10666000F0405395C9F77EF41F16BA0B620B730BFB
:10667000840BBAF09150A1F0FF0FBB1F661F771F6C
:10668000881FC2F70EC0BA0F621F731F841F48F421
:10669000879577956795B795F7959E3F08F0B3CFA7
:1066A0009395880F08F09927EE0F97958795089591
:1066B000E1D158F080E891E009F49EEFE2D128F0B2
:1066C00040E851E059F45EEF09C0ACC16DC2E92F5A
:1066D000E07831D268F3092E052AC1F3261737076F
:1066E0004807590738F00E2E07F8E02569F0E02535
:1066F000E0640AC0EF6307F8009407FADB01B90110
:106700009D01DC01CA01AD01EF935DD0F2D10AD049
:106710005F91552331F02BED3FE049E450FD49EC0A
:1067200063CF0895DF93DD27B92FBF7740E85FE39C
:106730001616170648075B0710F4D92F40D29F930F
:106740008F937F936F9349D3E0EAF0E06ED1D1D17C
:106750002F913F914F915F9175D2DD2349F0905871
:10676000A2EA2AED3FE049EC5FE3D0785D274DDFF8
:10677000DF91BFC102D280F09F3740F491110EF437
:1067800014C260E070E080E89FE3089526F01B16D5
:10679000611D711D811D1BC135C1EFD008F481E061
:1067A000089577D1E395B6C10CD0A3C16AD140F06A
:1067B00061D130F021F45F3F19F003C15111F5C1EF
:1067C00031C1B9D198F39923C9F35523B1F3951B7E
:1067D000550BBB27AA2762177307840738F09F5F02
:1067E0005F4F220F331F441FAA1FA9F333D00E2E71
:1067F0003AF0E0E830D091505040E695001CCAF7DE
:1068000029D0FE2F27D0660F771F881FBB1F2617A2
:1068100037074807AB07B0E809F0BB0B802DBF0175
:10682000FF2793585F4F2AF09E3F510568F0C9C07B
:10683000BCC15F3FECF3983EDCF386957795679596
:10684000B795F7959F5FC9F7880F911D9695879526
:1068500097F90895E1E0660F771F881FBB1F621745
:1068600073078407BA0720F0621B730B840BBA0B03
:10687000EE1F88F7E095089504D06894B11195C192
:10688000089561D188F09F5790F0B92F9927B7519B
:10689000A0F0D1F0660F771F881F991F1AF0BA95E4
:1068A000C9F712C0B13081F07FD1B1E008957CC149
:1068B000672F782F8827B85F39F0B93FCCF38695DA
:1068C00077956795B395D9F73EF490958095709537
:1068D00061957F4F8F4F9F4F0895E89409C097FBB4
:1068E0003EF490958095709561957F4F8F4F9F4FA7
:1068F0009923A9F0F92F96E9BB279395F6958795EB
:1069000077956795B795F111F8CFFAF4BB0F11F4AD
:1069100060FF1BC06F5F7F4F8F4F9F4F16C0882354
:1069200011F096E911C0772321F09EE8872F762F8A
:1069300005C0662371F096E8862F70E060E02AF0CB
:106940009A95660F771F881FDAF7880F96958795B7
:1069500097F9089512D180F09F3740F491110EF00D
:1069600024C160E070E080E89FEB089526F41B16D8
:10697000611D711D811D2BC045C0990F0008550F69
:10698000AA0BE0E8FEEF16161706E807F907C0F0B5
:1069900012161306E407F50798F0621B730B840BBD
:1069A000950B39F40A2661F0232B242B252B21F497
:1069B00008950A2609F4A140A6958FEF811D811D37
:1069C000089597F99F6780E870E060E00895882354
:1069D00071F4772321F09850872B762F07C0662318
:1069E00011F499270DC09051862B70E060E02AF0D9
:1069F0009A95660F771F881FDAF7880F9695879507
:106A000097F908959F3F49F0915028F4869577951E
:106A10006795B7959F5F80389F4F880F96958795AC
:106A200097F908959FEF80EC0895DF93CF931F931C
:106A30000F93FF92EF92DF927B018C01689405C067
:106A4000DA2EEF01FFD0FE01E894A5912591359152
:106A500045915591AEF3EF01D8DDFE019701A801F4
:106A6000DA9479F7DF90EF90FF900F911F91CF911B
:106A7000DF91089500240A941616170618060906D1
:106A8000089500240A9412161306140605060895A4
:106A9000C9CF59D0E8F3E894EFEFBB273FE048ECCB
:106AA0005FE76B3D73078407950708F1FF279F5742
:106AB000B25A6A4D7F40894CF04032F4BE5565426F
:106AC000704F8643FF4F0894EE1F915030F0BB0F7C
:106AD000661F771F881FFF1FEBCF9EE7882332F0CA
:106AE000BB0F661F771F881F9A95C1F79395E09596
:106AF00089CF092E0394000C11F4882352F0BB0FA8
:106B000040F4BF2B11F460FF04C06F5F7F4F8F4FC5
:106B10009F4F0895EF93E0FF06C0A2EA2AED3FE001
:106B200049EC5FEB72DDE5DF0F90039401FC9058B8
:106B3000EDECF0E063C157FD9058440F551F59F03C
:106B40005F3F71F04795880F97FB991F61F09F3F5A
:106B500079F087950895121613061406551FF2CF83
:106B60004695F1DF08C0161617061806991FF1CFD3
:106B700086957105610508940895E5DFA0F0BEE7EC
:106B8000B91788F4BB279F3860F41616B11D672F1C
:106B9000782F8827985FF7CF869577956795B11DF1
:106BA00093959639C8F30895E894BB27662777270D
:106BB000CB0197F90895E1DE08F48FEF08959B016A
:106BC000AC0160E070E080E89FE3EECDBCDF58F1FF
:106BD0009E5758F19851A0F0E9F0983020F5092E11
:106BE0009927660F771F881F991F0A94D1F712C043
:106BF000062E672F782F8827985F11F4000C07C0A6
:106C0000993FB4F38695779567959395D9F7611D6C
:106C1000711D811D3EF490958095709561957F4F13
:106C20008F4F9F4F08956894C0CFBECF0BD061CFD8
:106C300021DF28F026DF18F0952309F0C2CEF2CE2E
:106C40001124B3CF78DFA0F3959FD1F3950F50E0D7
:106C5000551F629FF001729FBB27F00DB11D639F0E
:106C6000AA27F00DB11DAA1F649F6627B00DA11DB4
:106C7000661F829F2227B00DA11D621F739FB00D5A
:106C8000A11D621F839FA00D611D221F749F3327CA
:106C9000A00D611D231F849F600D211D822F762F63
:106CA0006A2F11249F5750408AF0E1F088234AF060
:106CB000EE0FFF1FBB1F661F771F881F91505040AC
:106CC000A9F79E3F510570F07CCE6FCF5F3FECF38C
:106CD000983EDCF3869577956795B795F795E79598
:106CE0009F5FC1F7FE2B880F911D9695879597F9A9
:106CF000089529DFE0F09E37D8F09639B8F49E3831
:106D000048F4672F782F8827985FF9CF8695779575
:106D1000679593959539D0F3B62FB1706B0F711DB0
:106D2000811D20F4879577956795939550CE6ACE0F
:106D30003CCF9F93AEDE0F9007FCEE5FEBCE11F4DD
:106D40000EF470CE5FCEFFDED0F39923D9F3CEF3ED
:106D50009F57550B87FF4BD056959795B0E020F481
:106D6000660F771F881FBB1F1F930F93002490018E
:106D7000A0018001F001A0E80E0F1F1F0A1E511D87
:106D8000601B710B8009B50B48F4600F711F801DEB
:106D9000B51F0E1B1F0B0A0A510907C02E0F3F1FFC
:106DA0004A1F0E0F1F1F0A1E511D660F771F881FD7
:106DB000BB1FA695F795E795F8F60617170708067F
:106DC0005B07211D311D411D0F911F91B901842FBA
:106DD0009158880F9695879508959B01AC0126CF11
:106DE000CCDE20F09F3708F4E0CEF1CD0BCE9150F1
:106DF0005040660F771F881FD2F708959F938F9397
:106E00007F936F93FF93EF939B01AC010FDFEF91A3
:106E1000FF910BDE2F913F914F915F9107CF991B0F
:106E200079E004C0991F961708F0961B881F7A9581
:106E3000C9F780950895A1E21A2EAA1BBB1BFD017C
:106E40000DC0AA1FBB1FEE1FFF1FA217B307E40749
:106E5000F50720F0A21BB30BE40BF50B661F771FA1
:106E6000881F991F1A9469F7609570958095909581
:0E6E70009B01AC01BD01CF010895F894FFCF46
:00000001FF
